:1000000089C30000A3C30000A1C300009FC3000078
:100010009DC300009BC3000099C3000097C300006C
:1000200095C3000093C300000C9412220C94CE20C0
:100030000C943C248BC3000089C3000087C30000DC
:1000400085C3000083C3000081C300007FC300009C
:100050007DC300000C94FE2379C3000077C3000029
:1000600075C3000073C3000071C300006FC30000BC
:100070006DC300006BC3000069C3000067C30000CC
:1000800065C3000063C3000061C300005FC30000DC
:100090005DC300005BC3000059C3000057C30000EC
:1000A00055C3000053C3000051C30000E4045805C9
:1000B000EC04B604BA04F004BD04F304FE04C8045E
:1000C0004E05CC040205D00406053005D4040A050B
:1000D0003A05DA0410051A05C104F704C404FA0449
:1000E000DF041505260546054805B204E804610548
:1000F0008204E205EC05B005B505BA05BF05C405E7
:10010000C905CE05D305D805DD05A106A106D4068F
:10011000D40651076F076C086C087407E807F907E5
:10012000F907EC05B005B505BA05BF05C405C90555
:10013000CE05D305D805DD05FC182319DD1A2319D2
:10014000DD1A6E199019DD1A921AA21A0A310D31B0
:1001500013310C310F311231113105010980A10128
:10016000850319012AB700150126B70095017510FE
:100170008100C0050C0901A101850419012AA00212
:10018000150126A002950175108100C00501090620
:10019000A1018506050719E029E715002501950845
:1001A000750181020507190029EF1500250195F059
:1001B000750181020508190129059505750191024E
:1001C000950175039101C005010902A1010901A171
:1001D00000050919012908150025019508750181F7
:1001E000020501093009311581257F9502750881C5
:1001F0000609381581257F950175088106050C0AC9
:1002000038021581257F950175088106C0C00660FA
:10021000FF0961A1010962150026FF0095207508FC
:1002200081020963150026FF00952075089102C020
:1002300005010906A101050719E029E715002501B7
:10024000950875018102950175088101050719005E
:1002500029FF150026FF009506750881000508197D
:100260000129051500250195057501910295017576
:10027000039101C009027400040100A0FA090400FE
:1002800000010301010009211101000122440007BE
:1002900005810308000109040100020300000009B0
:1002A000211101000122220007058303200001071C
:1002B00005040320000109040200010301020009F2
:1002C00021110100012247000705820310000109E6
:1002D0000403000103000000092111010001226D47
:1002E000000705850320000112010002000000083C
:1002F000973276490001010203011A0339004200D6
:10030000340033004F002F00420034007A006700B1
:1003100067005100000016034500720067006F007F
:1003200064006F007800200045005A000000280398
:100330005A0053004100200054006500630068002B
:100340006E006F006C006F006700790020004C00A9
:100350006100620073000000040309043500E3003B
:10036000E000E100350000001E00140004001D0044
:10037000340001001F001A0016001B00454E2A0021
:100380002000080007000600E200280021001500F8
:10039000090019004F000100220017000A000500A3
:1003A0000000E300500061520000E2000000225013
:1003B0004F0062520000E7000000010023001C0013
:1003C0000B0011000000E600240018000D001000D2
:1003D000C152010025000C000E0036002F002C0039
:1003E000260012000F00370030002B0027001300FA
:1003F00033003800300001002D0031003400C152BC
:1004000081520000290001000100010001000000EC
:100410003A001E024A002E002E00427E3B001F02C0
:1004200021022D00010001003C004D0026022E0299
:10043000010028783D0030024F0130000100417E6C
:100440003E0031023500500100002178010001001A
:100450000000010000000100010001000000010097
:10046000000020783F0052005000240200000100EC
:100470004000240051001E000100007E41002500C4
:1004800052001F0037002378420026004F00200052
:1004900027002478430025022E0231002E0001009F
:1004A00044004500010001000100000001000100BE
:1004B0000100010001000000010001000100010035
:1004C0000100010001000100CF0001000100010056
:1004D0000100CD00CE000100D100010001000100AB
:1004E000D0000100D2000100010001000100010064
:1004F00000000100010001000000010000000100F7
:1005000001000100000001000000010001000100E5
:1005100001000100000001000100010001000100D4
:10052000A9000100010001000100AC00AA00B60012
:10053000010001000100AB00A80001000100010062
:100540000100010001000100007C0100AE0001007B
:1005500001000000002010300050406000312141B7
:100560000061517100120222004232520072628216
:1005700000130323005343630014042400645474E1
:1005800000150525004535550075658500160626BC
:1005900000463656001707270047375700281838F7
:1005A000005848680039294900695979001A0A2A0F
:1005B000004A3A5A01201030015040600131214177
:1005C00001615171011202220142325201726282B2
:1005D000011303230153436301140424016454747D
:1005E0000115052501453555017565850116062658
:1005F0000146365601170727014737570128183893
:10060000015848680139294901695979011A0A2AAA
:10061000014A3A5A000101010101010101010202EE
:1006200002020202020202030303030303030304A0
:10063000040404040404050505050506060606066B
:10064000070707070708080808090909090A0A0A25
:100650000B0B0B0C0C0C0D0D0D0E0E0E0F0F0F10C7
:100660001011111112121313141415151616171751
:10067000181819191A1A1B1B1C1D1D1E1E1F2020BD
:10068000212222232424252626272829292A2B2C07
:100690002D2D2E2F30313232333435363738393A2A
:1006A0003B3C3D3E3F404142434445464748494A22
:1006B0004C4D4E4F50515354555658595A5B5D5EF0
:1006C0005F616264656668696B6C6D6F707273758B
:1006D00077787A7B7D7E8082838587888A8C8E8FEF
:1006E00091939596989A9C9EA0A2A3A5A7A9ABAD1D
:1006F000AFB1B3B5B7BABCBEC0C2C4C6C9CBCDCF0B
:10070000D1D4D6D8DBDDDFE2E4E7E9EBEEF0F3F5B8
:10071000F8FAFDFF11241FBECFEFDAE0DEBFCDBF38
:1007200012E0A0E0B1E0E6E1FBE602C005900D9228
:10073000A239B107D9F726E0A2E9B2E001C01D92C3
:10074000A038B207E1F7FFD40C94893559CCA0E06A
:10075000B0E0EDEAF3E00C942234FC012481222382
:1007600009F4ECC48C0161E00E941230EC01F80144
:100770008581C234F8E7DF0709F46DC030F4C03278
:1007800038E7D30709F467C07BC0C1159EE7D907D6
:1007900009F43FC0C130EEE7DE0709F071C08823DD
:1007A00009F4BFC09091A40281E0890F8770987FFF
:1007B000853020F4892B8093A40202C09093A40278
:1007C0008091A4028770FFEF8F9FC001112495953F
:1007D00087959595879599279093890080938800B0
:1007E00090938B0080938A0090938D0080938C006F
:1007F0004091A4025091A5026091A6027091A702B7
:100800008FE090E00E94F1348091C7020E94F7309F
:1008100088C0882309F485C08091A40283FB222725
:1008200020F991E0922790FB83F98093A402992309
:1008300029F040E060E080E00E94672A4091A40235
:100840005091A5026091A6027091A7028FE090E0FE
:100850000E94F13466C0882309F45DC180912E04A2
:100860008F3F51F410922E040E94A11540E060E0E9
:1008700080E00E94672A4FC18FEF80932E044EC004
:10088000C0342EE7D207F9F028F4C5349EE4D90726
:1008900051F047C0C134EEE7DE07E1F0C234FEE7B5
:1008A000DF0719F13EC0811107C089E20E943A2F8B
:1008B00080E00E943D2E2FC180E00E94482E89E2F8
:1008C0000E94692F28C1882309F425C181E00E9474
:1008D000A71521C1882309F41EC181E00E94A71534
:1008E0004FEF6FEF85E890E00AC0882309F413C149
:1008F00081E00E94A7154EEE6FEF87EC90E00E941A
:10090000BC1509C180912904837011F410921F0154
:10091000809129048C7F8160809329040E94A11515
:10092000FAC0F8019581992309F407C19E01305757
:100930002332310508F0DBC084E090E00E94CB3424
:100940009093280680932706FE01E150F047E2329B
:10095000F10520F4EA5AFF4F0C946D35809127067B
:100960008160ACC0809128068860B4C08091270661
:100970008260A4C08091270620C0809127068860ED
:100980009DC0809128061EC0809128068260A2C06A
:1009900080912706806192C08091270680628EC078
:1009A0008091270680648AC00E940D2E80912706C0
:1009B000806884C080912706886084607FC08091B1
:1009C00028068260816086C0809127068E7F76C06F
:1009D00080912806877F7EC0809127068D7F6EC01C
:1009E0008091270620C080912706877F67C080916D
:1009F00028061EC0809128068D7F6CC08091270636
:100A00008F7E5CC0809127068F7D58C0809127061D
:100A10008F7B54C00E940D2E809127068F774EC089
:100A200080912706877F8B7F49C0809128068D7F24
:100A30008E7F50C08091270682FB222720F991E00B
:100A4000922790FB82F990FB83F938C080912806A9
:100A5000982F909591708E7F892B90FB81F93AC0E9
:100A60008091270686FB222720F991E0922790FBB0
:100A700086F924C00E940D2E8091270687FB22272D
:100A800020F991E0922790FB87F918C061E001C03E
:100A900060E08EE090E00E94DF341EC08091270667
:100AA00084FB222720F991E0922790FB84F906C06D
:100AB00080912706982F909590FB80F980932706C8
:100AC0000BC08091280683FB222720F991E0922712
:100AD00090FB83F980932806609127067091280681
:100AE00084E090E00E94F9340E940D2E14C08091A1
:100AF0009E04C6312CE7D20709F071C08A7A91E0D2
:100B000009F490E090939402811116C389E20E9447
:100B10009C240E94611D80917304877009F40EC3A8
:100B2000F8018581882309F409C38091280682FF92
:100B300005C382E00E94B61D01C3C631FCE7DF0792
:100B400009F4ECC280919E048272FE01E054F847E1
:100B5000ED30F10508F04BC0E858FF4F0C946D35AF
:100B6000882329F00E949E27D6CF8823D9F30E949C
:100B7000A727D1CF882329F00E948C27CCCF8823A8
:100B8000D9F30E949527C7CF882329F00E947427A4
:100B9000C2CF8823D9F30E948027BDCF882329F0B4
:100BA0000E945C27B8CF8823D9F30E946827B3CF6F
:100BB000882329F00E944827AECF8823D9F30E94CA
:100BC0005227A9CF80912904837011F010921F0140
:100BD000809129048C7FA0CE0E94B1279CCF827285
:100BE000FE01E052F847EB30F10508F4A1C29E0186
:100BF000205E324520323105A8F4911115C0CF7125
:100C000081E090E09C0102C0220F331FCA95E2F7F9
:100C1000E901622F83E090E00E94DF348C2F0E9474
:100C2000E12D79CF9923B9F1C3303CE7D307E1F047
:100C300040F4C1159CE7D90789F0C130DC47D1F0F9
:100C40002AC0CB35FCE7DF0719F1CC352CE7D207FA
:100C5000B9F0CA35DC47F9F481E01BC081E00E949D
:100C6000D7300E94CC2357CF6FEF7FEF80E090E02A
:100C70000E94F93480E00E94D7300E94C1234BCFFC
:100C80008091280682FB882780F991E0892701C09E
:100C900080E00E94CD1DF8018581C081D18188232B
:100CA00049F0CE010E94232DF82E682FCE010E941C
:100CB000922D04C0CE010E945E2DF82EBE018F2D14
:100CC0000E94281C0E94451CF82EC92FD82EF8011E
:100CD000D581E680E2949FE0E922809173048770D9
:100CE00001F1DD23F1F08C2F807F803469F080E208
:100CF0008F0D8830B0F08C2F807E803229F4F1E0A7
:100D0000FF1578F4EE2069F08091280682FF09C073
:100D100082E00E94B61D809173048770CC24C39436
:100D20008111C12CBC2EB2948FE0B8228B2D90E0A3
:100D30008C30910508F0D0C1FC01EB57FF4F0C94AB
:100D40006D358C2F807FCF70882311F0C295C07FC6
:100D5000DD23B9F0CC2309F4ADC180E28F0D8830DA
:100D600010F0D11006C090919E04C92BC0939E0430
:100D700005C090917504C92BC09375040E94611D34
:100D800099C18F2D0E943A2FCC2309F4A5C180E28E
:100D90008F0D883088F1DD2079F1C0959091750430
:100DA000C923C09375042BC08C2F807FCF708032F5
:100DB00011F0C295C07F8F2DDD2029F021E0D216E1
:100DC00009F44CC055C08091280682FD1BC0DD236C
:100DD00069F0CC2339F090919E04C92BC0939E04F6
:100DE0000E94611D80E00E94692F76C180E00E9410
:100DF0003A2FCC2309F470C18C2F0E945A1D0E94F7
:100E0000611D6AC1DD2381F0EE20B1F131E0E31212
:100E100063C1909174048C2F8923C81709F45CC1B5
:100E2000C92BC093740458C1E11056C18C2F0E9485
:100E3000522E809174049C2F982329F09C2F90951A
:100E4000892380937404209195028C2F822309F4C6
:100E500043C1C0952C23209395023EC1DD2329F088
:100E600081E08E1508F438C107C0E11035C115C006
:100E7000DD2331F0E1101EC18C2F0E94592E2CC1B0
:100E8000EE2059F0893309F024C19FEFE7EEF3E03B
:100E90009150E040F040E1F71AC18C2F0E94522E91
:100EA0001BC18C2F86958695837019F0813061F077
:100EB00013C1DD2321F08F2D9C2F937002C080E0A1
:100EC00090E00E94FA240FC1DD2321F08F2D9C2F8A
:100ED000937002C080E090E00E94D32404C16D2F83
:100EE0008F2D0E94632EFFC08C2F8370A9F5D11126
:100EF000F7C04F2D429546954770440F440F8F2DF4
:100F00008F7090E09C01042E01C0220F0A94EAF732
:100F1000F4FE08C08FE090E001C0880F4A95EAF720
:100F2000809501C080E0C695C695C370C23069F057
:100F300088F49091C602C13019F0822B892302C037
:100F4000922B892B0E94E12DCBC0822B9091C6025F
:100F50008927F8CF822BF6CFDD2319F08C2F8170F3
:100F600001C08695882309F4BBC04F2D4295469554
:100F70004770440F440F8F2D8F7090E09C01042E1A
:100F800001C0220F0A94EAF7F4FE08C08FE090E057
:100F900001C0880F4A95EAF7809501C080E0C695A8
:100FA000C695C370C23059F078F49091C702C13031
:100FB00019F0822B892309C0922B892B06C0822B22
:100FC0009091C702892701C0822B0E94C72D88C03B
:100FD000CF70DD2339F08C2F0E94D72D8F2D0E94EA
:100FE000592E7EC08F2D0E94522E8C2F0E94CC2D08
:100FF00077C08F2D22EFD21669F12D1538F030EF22
:10100000D31659F091EFD91601F150C0E3EFDE1677
:1010100041F1F4EFDF16A9F049C0DD2369F0E110DA
:101020005BC0CF7181E090E001C0880FCA95EAF7FC
:101030009091C70289271FC021E02E1508F44CC0EB
:10104000F0CF8091280682FD19C0DD2329F08C2F76
:101050008F711FC0DD23D9F38C2F8F710E94CC2D8F
:101060003BC0DD2339F0CF7181E001C0880FCA9504
:10107000EAF701C080E00E94C72D2EC0DD2361F099
:101080008C2F8F7198E0899F900111242360209309
:1010900073040E94D72D20C081E00E94B61DE1E0BC
:1010A000EE15D0F482E00E94B61D16C0DD2321F0BB
:1010B000EE2069F28F2D97CEEE2071F2893349F43C
:1010C000FFEF27EE33E0F15020403040E1F700C061
:1010D00000008F2D0E943A2F88EF8B0D843018F47A
:1010E0000E94212516C0CC20A1F08091730480FDC0
:1010F00010C0F80115828695869586950E94D72D99
:10110000C80125DB809173048695869586950E949B
:10111000CC2D60E0C8010E94123010C08091940272
:10112000811104C089E20E946E24F3CC85E3FBCFD9
:10113000EF56FF4F0C946D3585E3E9CCCDB7DEB7A4
:10114000E9E00C943E34A3E7B0E0E9EAF8E00C945F
:10115000193485B7806885BF85B7806885BF84B737
:10116000877F84BF0FB6F894A8958091600088614E
:1011700080936000109260000FBE90E080E80FB690
:10118000F89480936100909361000FBE81E080939A
:101190001B0185EF9AE190939302809392020E9443
:1011A00012210E94B8218091E20084608093E200C5
:1011B00078948091F2038823A1F01091E9001F70C8
:1011C0009091EC00892F817090FD80E8182B10928F
:1011D000E9008091E80083FD0E9415181F701093AC
:1011E000E90082E084BD93E095BD9AEF97BD8093BE
:1011F0006E000E941E3290E09093110180931001C6
:101200000E9499310E94F931E6E9F2E0A8EAB2E0E1
:1012100011921D9222E0E43AF207D1F780E090E0CB
:101220000E94CB34833E9E4F09F443C063EE7EEFB1
:1012300080E090E00E94F93460E082E090E00E945B
:10124000DF3481E08093C60261E083E090E00E9499
:10125000DF3460E074E184E090E00E94F9340E94A1
:101260006C2A1092A4021092A5021092A60210926B
:10127000A70284E08093A4024091A4025091A502A9
:101280006091A6027091A7028FE090E00E94F13475
:1012900040E050E0BA0183E190E00E94F13448E080
:1012A00050E067E170E089E294E00E94D03410924F
:1012B000310482E090E00E94BE348093B60284E064
:1012C00090E00E94CB3490932806809327060E94DA
:1012D000C81F4FEF53EF81E0415050408040E1F78D
:1012E00000C000000E94C81F8091A80280FF08C0B3
:1012F0006FEF7FEF80E090E00E94F9340E94CC23F2
:1013000083E090E00E94BE340E94E12D8091C702EC
:101310000E94F7300E941A2610920004E9E1F4E0DE
:101320008FEF9FEF81939193A4E0E932FA07D1F711
:1013300010922F06E8E4F6E088E596E02FEF3FEF05
:10134000219331938E179F07D9F781E08093310461
:1013500048E050E067E170E089E294E00E94AE343A
:1013600010923104809129048C7F11F40E946C2A20
:1013700089EA8093800089E08093810024982C98EA
:101380003F98479A54985C9A55985D9A6E98769AC9
:10139000569A8FE090E00E94C6346093A402709346
:1013A000A5028093A6029093A70267701FEF169F75
:1013B000B00111247595679575956795772770939A
:1013C00089006093880070938B0060938A0070930B
:1013D0008D0060938C005E980E94EA300E94E63097
:1013E0000E94E2308FEF90E0909389008093880014
:1013F00090938B0080938A0090938D0080938C0053
:101400000E94F430BFEFE0E7F2E0B150E040F0407E
:10141000E1F700C000000E94F1302FEF30E742E01A
:10142000215030404040E1F700C000000E94EE3003
:101430005FEF80E792E0515080409040E1F700C0BC
:1014400000000E94EA30AFEFB0E7E2E0A150B04008
:10145000E040E1F700C000000E94E630FFEF20E727
:1014600032E0F15020403040E1F700C000000E941F
:10147000E2308091A4028770189FC00111249595D5
:1014800087959595879599279093890080938800F3
:1014900090938B0080938A0090938D0080938C00B2
:1014A0005E980E94EA300E94E6300E94E23080910D
:1014B0002904843B18F080E00E94A71584E091E0A5
:1014C00090932406809323068091F203853009F0DF
:1014D0006FC011E000E443E0F42E50E1E52E62E13C
:1014E000D62E8091F203853009F05CC08091F20322
:1014F000843009F437C00E94C52780915C068111B1
:101500000CC023D410922101809129048370809310
:1015100020010E947720F0921F0110935C06109228
:10152000290648E150E00FB6F894A8954093600072
:101530000FBE0093600083B7817F846083BF83B751
:10154000816083BF7894889583B78E7F83BF0FB601
:10155000F894A89580916000886180936000109253
:1015600060000FBE0E941E3290E0909311018093A4
:1015700010010E9499310E94F931E8EAF2E01192DB
:1015800086EB92E08E179F07D1F70E94C81FE8EA0A
:10159000F2E081918111B5C3A6EBB2E0AE17BF07AF
:1015A000C1F79FCF0E940D2E0E94212510925C064C
:1015B0000E94C81FE7EBF2E0AA96FFAFEEAFAA9732
:1015C000A8EAB2E091918D91892722E0E53CF207EB
:1015D00019F08823B9F305C0811103C00E9452207D
:1015E0009EC134E9232E33E0332E48E451E0AC961B
:1015F0005FAF4EAFAC9788EA92E0E0969FAF8EAFB8
:10160000E097F12CE096AEADBFADE0977D90E0960F
:10161000BFAFAEAFE097AA96EEADFFADAA97C08080
:10162000C724AE96CFAEAE97CC2009F45BC1610162
:10163000AC964EAC5FACAC97E12C66246394AE964E
:101640008FADAE97862109F43DC1872C8620A296E6
:10165000EFAEA297A396FFAEA3970E943024A59663
:101660009FAF8EAFA597F1E0A696FFAFA69791E04A
:10167000811001C090E0A7969FAFA797A2964FADAB
:10168000A297A3965FADA397A4966FADA497A596D6
:101690007FADA597A6968FADA6970E94383088207B
:1016A00051F0D2018C918F3F31F0AD968FAFAD9755
:1016B0009924939401C0912C092D10E080912F065C
:1016C000F801E80FF11D3997ACF188E0A82EB12C94
:1016D000A01AB10AB8016F5F7F4F615D794FA50114
:1016E00080E396E00E948035B801675F7F4F615DBF
:1016F000794FA50188E396E00E948035A501440F4B
:10170000551FB801660F771F675E7F4F615D794F88
:1017100088E496E00E948035B8016F5E7F4F615D7E
:10172000794FA50180E496E00E94803588E0891910
:1017300080932F0680912F0690E0AD96FFADAD9778
:10174000AF2FB0E09D01220F331F24563E4FAA0F4A
:10175000BB1FBD0163567E4F41E0480F9915C0F491
:1017600090E0FC01E15DF94FD9015C915183DB010F
:101770005C915187AD96BFADAD97B18B880F991F26
:10178000FC01E15DF94F128E118E91E0842FE4CFC0
:1017900080932F06882009F495C0809129048C7FBE
:1017A0008C3709F08FC0F20180818F3F09F48AC025
:1017B00078E4A72E71E0B72EE4E98E2EE3E09E2EAA
:1017C000A8961FAEA89790E09C01220F331FA90195
:1017D00044565E4FE2965FAF4EAFE297D901A356F3
:1017E000BE4FE496BFAFAEAFE49700E010E0F50166
:1017F000E00FF11F80818F3F09F44EC0A896BFAD66
:10180000A897BF110AC0E01208C0F601208130E29B
:10181000230F08F42FEF20833FC090E0E296EEAD57
:10182000FFADE297408150E0FC01EE0FFF1FE45650
:10183000FE4F2081421B5109E496AEADBFADE49747
:101840002C9130E0880F991FFC01E356FE4F8081F8
:10185000281B3109449FB001459F700D700D112464
:10186000229FC001239F900D900D1124860F971F7A
:101870000E94C62A893280F428E2382F231B08F4FC
:1018800020E0F401E00FF11F213108F020E1308168
:10189000320F08F43FEF30830F5F1F4F0630110502
:1018A00009F0A5CFA8964FADA8974F5FA8964FAF68
:1018B000A89756E0850E911C86E0A80EB11C4E300C
:1018C00009F093CFE394660C9FEF491A590AAFEFE2
:1018D000CA1ADA0AB6E0EB12B2CEAA96EEADFFADA6
:1018E000AA977082F394AA962EAD3FADAA972F5F68
:1018F0003F4FAA963FAF2EAFAA97AC964EAD5FADC5
:10190000AC974A5F5F4FAC965FAF4EAFAC9756E077
:10191000250E311C8EE0F81275CE0E9424240E9400
:10192000C527B0901C0610911D06C0901E060091A0
:101930001F06D090200610921D0610921E061092CF
:101940001F0610922006111103C0CC2009F449C0D3
:10195000E0901A06F0901B060E9430249C012E197C
:101960003F0990911506992309F4E6C12531310507
:10197000C0F19F3F19F09F5F90931506112361F00E
:101980000E947825111614F491E001C09FEF899F01
:10199000802D112480931D06CC2061F00E947825B3
:1019A0001C1414F09FEF01C091E0899F802D112439
:1019B00080931E0680911D06882399F0F0901E06E4
:1019C000FF2079F00E949B25811101C081E0809366
:1019D0001D068F2D0E949B25811101C081E08093FF
:1019E0001E06011103C0DD2009F449C0E09018066D
:1019F000F09019060E9430249C012E193F09909105
:101A00001606992309F49CC125313105C0F19F3F89
:101A100019F09F5F90931606002361F00E945825ED
:101A2000101614F491E001C09FEF899F802D1124BE
:101A300080931F06DD2061F00E9458251D1414F0CC
:101A40009FEF01C091E0899F802D11248093200693
:101A500080911F06882399F0F0902006FF2079F0EE
:101A60000E949B25811101C081E080931F068F2D6C
:101A70000E949B25811101C081E080932006809106
:101A80001C068B111AC080911D06882311F01813B3
:101A900014C080911E06882311F08C110EC0809115
:101AA0002006882311F0D81208C090911F069923B0
:101AB00031F081E0091304C002C081E001C080E080
:101AC00080FD15C080911D0681110FC080911E06FA
:101AD00081110BC080911F06811107C081E0909198
:101AE0002006911103C080E001C081E080FD0E94CA
:101AF0003025B0921C0610931D06C0921E0600935E
:101B00001F06D09220060E9421259091C5028917B8
:101B100021F08093C5020E9424248091F203843036
:101B200009F0D2CC8093E9008091E80082FFCCCC10
:101B30008091E80085FF23C00E94312181111DC0E2
:101B400080E2E82EF12C8E010F5B1F4F09C08091BF
:101B5000F100D8018D938D01B1E0EB1AF10869F025
:101B60008091E80085FDF3CF8091E8008B7780932A
:101B7000E8000E943121882399F391E001C090E0B0
:101B80008091E8008B778093E800992309F49CCC3E
:101B900022968FAD2297863009F495C020F58230C9
:101BA00009F492CCD0F4882399F1813009F0A5C0D2
:101BB0008093C80284E089A31EEF1AA3CE01819608
:101BC000BAD79091C7028091C602892B0E94FE2F3E
:101BD00095E099838A831B838CC0843031F18530F2
:101BE00009F471C08AC0893009F46DC030F48730BF
:101BF000C9F1883009F467C080C08A3009F465C033
:101C00008E3F09F07AC0898394E09A838B8371C0F8
:101C100019828DE0E7E2F1E0DE01129601900D926B
:101C20008A95E1F78EEF8E8764C08091C802882381
:101C300009F44ACC23968FAD2397811106C02496D0
:101C40008FAD24970E94CC2D3FCC81E090E024966C
:101C50000FAC249702C0880F991F0A94E2F70E94E4
:101C6000C72D32CC81E08093CA0223968FAD239793
:101C70008230E1F030F5882319F0813061F021C025
:101C800024968FAD2497882319F00E94F4301CCC41
:101C90000E94EA3019CC24968FAD2497882319F03E
:101CA0000E94F13011CC0E94E6300ECC24968FAD0C
:101CB0002497882319F00E94EE3006CC0E94E2306F
:101CC00003CC85E01BC084E019C023968FAD239719
:101CD00011E0811101C010E01093CA02811106C009
:101CE0000E94EA300E94E6300E94E2308BE0898355
:101CF0001A83CE0101961FD7E7CB8FEF0E944131A7
:101D0000E3CB8091F103882309F4EBCBE9BCD9BC88
:101D100009B400FEFDCF8091D8008F7D8093D8005C
:101D20008091E00082608093E0008091E00081FD7E
:101D3000FCCF0E940D2ED5CB232B09F01CCE51CE0B
:101D40002139314008F065CE9ACEA5E0B0E0EBEA4B
:101D5000FEE00C941934782E8091210187110DC07A
:101D600020912904237030E04091200150E081E06F
:101D70002417350719F480E001C081E08170809359
:101D80001E0180912E0490911D01981739F08093C7
:101D90001D0140E060E080E00E94672A86E1781241
:101DA00046C085E399E20E940F1709C0271508F481
:101DB00067C235E073125EC288E89CE2EDD7898382
:101DC00021C0A71508F450C2B1E07B1288C08091F1
:101DD0001C010E94BB279A83898360912A04709119
:101DE0002B0480912C040E949D2C162F072FF82E77
:101DF0004A815981541708F4CFC081E08983403368
:101E000008F0C8C080911C018F5F80931C0159812C
:101E100051118DC682E080931F0180911E018111B6
:101E200086C6711084C683E080931F0180C6871523
:101E300008F473C29AE079120EC080ED9BE208C0EC
:101E4000A71508F43EC2BBE07B1235C287EB9BE2CC
:101E50000E945E17B4CF971508F41FC2A4E07A124F
:101E6000B0CF80911C010E94BB279A838983E090A8
:101E70002B04D0902C0460912D0480E40E943E2B12
:101E8000F82EEA81F981FE1708F052C0A9810A2FC5
:101E900010E0F801E450FE4F908180911D018923EC
:101EA000D1F0F801EE0FFF1FE456FE4F6081F69E61
:101EB000B0011124E5E075956795EA95E1F7809109
:101EC0002A04680F7E2D8D2D0E949D2C472F282FD0
:101ED000C8010E946A2AB981BF5FB983D2CF7B163D
:101EE00008F44FC0E2E07E1286C080911C010E947F
:101EF000BB279A83898300912B0410912C04F090C6
:101F00002A046F2D702F812F0E949D2CE62ED72E34
:101F1000C82E60912D046F0D702F812F0E949D2C73
:101F2000162F072FF82EEA81F981FE1708F449C011
:101F300021E0298322C0E71508F4F4C280911C0136
:101F4000F7E17F1287C1882309F45EC280911C01EA
:101F50000E94BB279A83898390911E01911170C2C0
:101F60004091120150911301282F30E0421753077E
:101F700008F074C2B1E0B983EA81E03308F442CFDB
:101F800009C080911E01882329F040E060E080E0D4
:101F90000E94672A198236CF2981E22FF0E0DF0103
:101FA000A450BE4F8C9190911D01982331F02F2D9C
:101FB000402F612FCF010E946A2A39813F5F398308
:101FC00017CFA9818A2F90E0FC01E450FE4F3081A9
:101FD00020911D01232359F030FF04C02F2D402FE5
:101FE000612F03C02C2D4D2D6E2D0E946A2AB981C0
:101FF000BF5FB98398CFF3E07F1230C180911C019D
:102000000E94BB279A838983E0902B04D0902C04F4
:1020100060912D0480E40E943E2BF82E5A81898124
:10202000851728F53981032F10E0F801E450FE4FA1
:10203000908180911D018923B1F0F801EE0FFF1FFF
:10204000E356FE4F808182958F7060912A048F9DA8
:10205000600D11247E2D8D2D0E949D2C472F282F41
:10206000C8010E946A2A49814F5F4983D7CF91E016
:102070009983ECC0A71508F4B9C4BCE17B1609F438
:1020800053C1B71508F0BAC15FE1751609F456C21D
:10209000571508F4DCC38DE1781609F4F8C29EE107
:1020A0007912DCC080911E01882329F040E060E0B5
:1020B00080E00E94672A80911C010E94BB279B83BD
:1020C0004091FC035091FD036091FE037091FF036A
:1020D00080918B0390918C03A0918D03B0918E031E
:1020E00084179507A607B70708F0ADC060912A04CA
:1020F00070912B0480912C040E949D2C362E7A83A3
:10210000282E01E613E0A8E4B1E0BD83AC83ACE97E
:102110008A2EA1E09A2EAC80BD806501780132E064
:102120003983F701808181118AC3412C512C612CA4
:10213000D501ED915D01F0E0DF01A450BE4F8C911F
:1021400090911D01982331F0242D452D662DCF014E
:102150000E946A2AD6011596EC91F0E0DF01A450A6
:10216000BE4F8C9190911D01982331F0242D452D67
:10217000662DCF010E946A2AF7018181D7018D93D4
:102180007D01B981B150B983E1E0CE1AD108B11116
:10219000C8CFD80112968C91811155C3D12CE12C56
:1021A000F12CAC81BD811296EC91F0E0DF01A450DE
:1021B000BE4F8C9190911D01982331F02D2D4E2D05
:1021C0006F2DCF010E946A2AAC81BD811396EC91DC
:1021D000F0E0DF01A450BE4F8C9190911D01982337
:1021E00031F02D2D4E2D6F2DCF010E946A2A0E94B5
:1021F000A82A837091E009F090E0F80192830D5FC6
:102200001F4F2C813D812A5F3F4F3D832C838216D7
:10221000930609F080CF0E942C2B0091FC031091B3
:10222000FD032091FE033091FF03DC01CB01800F01
:10223000911FA21FB31F80938B0390938C03A093D5
:102240008D03B0938E0341E049835B81503308F4E2
:10225000D9CDA0CE28E1721609F413C180911C01DA
:102260008F5F80931C01D6CD27E072129FCD81E253
:102270009CE2A4CD46E07412F1CF84E59CE29ECDB1
:1022800058E0751203C085E09CE205C089E0781231
:10229000E5CF8AEE9BE278D692CD90E1791203C029
:1022A00083ED99E2D5CD9715C0F0ADE07A12C8CD97
:1022B00086E09AE283CDECE07E12D0CF8FE09AE206
:1022C0007DCDFEE07F1203C08DEF99E277CD2FE048
:1022D0007212C4CF82EE99E271CD33E1731203C062
:1022E00084E49AE2B5CD371560F041E1741203C081
:1022F00087EF9AE2D0CF52E17512B0CF87E59AE22C
:10230000CACF84E1781203C085EA99E24CCD95E109
:102310007912A4CF83E799E246CDA2E27A12AACE3F
:1023200086E49BE2D0D44BCD80911C01811123C067
:102330002091CB023091CC023D832C830E9430242B
:1023400040912D0420E431E0241B31094C815D8152
:10235000841B950B2817390770F480E30E94BD2A6F
:1023600090E090931701809316010E94302490937F
:10237000CC028093CB0280911C010E94BB27192FB5
:10238000A0911601B0911701BD83AC8390E0A8170E
:10239000B90770F1812F90E0A817B90748F5FD0142
:1023A000E450FE4F908180911D01892309F10E9424
:1023B000A82A81FD0BC00E94A82A082F80E80E944D
:1023C000BD2A7FE7780F80912C0403C080E070E085
:1023D00000E0602F0E949D2C472F282F8C819D812B
:1023E0000E946A2A81E390E090931701809316017E
:1023F000B1E0B983103308F405CDCCCDE9E17E120C
:102400009ACD80EA9BE2DACC60912D0420E1620F44
:1024100008F46FEF8091FC039091FD030E941F2B45
:102420006AE070E00E940534892B09F08FCD80E3CB
:102430000E94BD2A90E0909313018093120186CDF3
:102440004A815981541708F095CD60911D01898109
:102450000E94102739813F5F3983F2CFAA818A2FEA
:1024600090E04817590708F085CD60911D01842F31
:102470000E94102781E390E0909313018093120152
:1024800079CD81111AC060912D0420E1620F08F40A
:102490006FEF8091FC039091FD030E941F2B65E07C
:1024A00070E00E940534892B41F480E30E94BD2A2C
:1024B00090E0909315018093140180911C010E947B
:1024C000BB279A83898390911E01992371F02A81F9
:1024D0003981321708F04ECD60911D0189810E942B
:1024E000F326F981FF5FF983F2CF409114015091F7
:1024F0001501282F30E04217530708F43BCDAA817D
:102500008A2F90E04817590708F034CD60911D01DB
:10251000842F0E94F32681E390E09093150180932D
:10252000140128CD3AE1731203C08FE79BE246CC39
:102530004BE1741293CE85E69BE240CC80911C0166
:102540000E94BB271C0180911E01882361F040E09E
:1025500060E080E00E94672A84E5E4E9F3E0DF01BF
:102560001D928A95E9F780911C0181111BC0E091B1
:102570009003F0919103FD83EC830E9430242C8121
:102580003D81821B930B21E08931910508F420E005
:1025900020938F03499730F00E9430249093910349
:1025A0008093900378E4C72E71E0D72EE4E9EE2EF5
:1025B000E3E0FE2EF2EE8F2EF3E09F2E512C00E092
:1025C00010E0F601E00FF11F30813983321508F475
:1025D00044C0331508F041C05394432F50E05D834D
:1025E0004C83FA01E450FE4F908180911D018923B4
:1025F00009F433C05701A00EB11ED5016C90262DF1
:1026000035E5231B08F420E0422E40912B0449833A
:102610002AEA562D250F08F42FEF822F92E0299FEA
:10262000800D112460912C048E5F0E943E2B6AEA7B
:10263000641979810E949D2C472F282F8C819D81C0
:102640000E946A2A80918F03882339F0262D31E079
:10265000231B08F420E0D5012C930F5F1F4F063099
:10266000110509F0AECF8E149F0451F0B6E0CB0EE9
:10267000D11CE6E0EE0EF11CF4E0F51508F09FCF5A
:1026800021E029833FE2331508F0BCCB83CC409195
:102690005D0350915E0360915F03709160038091D0
:1026A000FC039091FD03A091FE03B091FF038417FA
:1026B0009507A607B70708F46DCC80911E0181111C
:1026C00007C080911C010E94BB27092F89834DC040
:1026D00040E060E080E00E94672AEDECF2E0FD83DC
:1026E000EC8310E30E94A82A81FF09C0AC81BD8160
:1026F0001C9211961C92119712961C9212C00E9465
:10270000A82A082F80E80E94BD2A7FE7780F602F53
:1027100080912C040E949D2CEC81FD81608371834B
:10272000828311502C813D812D5F3F4F3D832C834F
:102730001111D8CFC6CF3981832F90E0FC01E4502E
:10274000FE4F308120911D01232361F0FC01EE0F2B
:10275000FF1FE80FF91FE353FD4F22814181608184
:102760000E946A2A49814F5F49835981501718F3A3
:1027700081E08983003308F01982003308F442CBEA
:1027800020E010E001501109822F90E0801791079E
:10279000C4F4DC01AA0FBB1FA80FB91FA353BD4F80
:1027A0000196FC01EE0FFF1F8E0F9F1FFC01E353EC
:1027B000FD4FC080D180E280CD92DD92EC922F5F00
:1027C000E3CF0E94A82A7801EE0CFF1C81FF09C00C
:1027D0000E0D1F1DF801E353FD4F1082118212826E
:1027E00015C00E94A82A8A8380E80E94BD2A7FE73C
:1027F000780F6A8180912C040E949D2C0E0D1F1D64
:10280000F801E353FD4F6083718382830E942C2B78
:102810000091FC031091FD032091FE033091FF0312
:10282000DC01CB01800F911FA21FB31F80935D03BA
:1028300090935E03A0935F03B0936003E3CA422CBE
:102840005A80632C75CCD22CEA80F32CAACCA0E25F
:102850007A12C6C060902C0483E0689EA001112407
:1028600056954795569547955D834C839C819983F2
:10287000862C912C8FEF90E0B4010E945A35362EB1
:1028800080911E01882371F040E060E080E00E94AA
:10289000672A84E5E4E9F3E0DF011D928A95E9F710
:1028A00010929303809192038F5F8093920334E997
:1028B000E32E33E0F32E48E4A42E41E0B42E5AE98F
:1028C000452E53E0552EEC81FD818E1A9F0A87011B
:1028D0006501212C21100CC080919303811108C047
:1028E0000E949734853595401CF4D7016C920CC03A
:1028F000F8018081882341F0861530F4909192038D
:10290000391202C081508083D601EC91EF3F29F14A
:10291000D8012C91F0E0B981B21790F430E04C81ED
:102920005D81241B350B249FC001259F900D349F92
:10293000900D1124B4010E940534262F462D0AC0A3
:10294000629EC00111246C817D810E940534462F56
:1029500020E060E0CF010E946A2A239456E0C50E71
:10296000D11C0A5F1F4F8EE02812B4CF9FEFE91AE7
:10297000F90AAFEFAA1ABA0A4E145F0409F0A7CFFA
:1029800080919203381202C01092920380919303B7
:102990008F5F8D3118F480939303FCCA10929303D8
:1029A0002CED33E08DE048EE53E09FEF960DA2EE64
:1029B000B3E0F9018D3021F46C91661201C09C9353
:1029C0006081661510F090836682319611964A17E1
:1029D0005B0781F78150265031098111E8CFDACAAF
:1029E000B1E27B123BCC88E59BE29CCCE8E27E1214
:1029F0000BC062EB78E205C034E273122FCC6CE1BD
:102A000079E280E0C5D0DBC9E71508F432C0F5E211
:102A10007F120BC08091000421E0482F421B08F474
:102A200040E0842F64EE78E2EDCFF71570F023E2FA
:102A30007212E2CF8091000421E0382F321B08F49B
:102A400030E0832F6CE179E2DDCF46E2741203C0FF
:102A500064EE78E2D6CF57E2751200CC8091000484
:102A600021E0582F521B08F450E0852F62EB78E2EA
:102A7000C9CF8BE278120BC08091000421E0482F6F
:102A8000421B08F440E0842F64E878E2BBCF87154E
:102A9000A0F099E279120BC08091000421E0382F58
:102AA000321B08F430E0832F6AE978E2ABCFAAE268
:102AB0007A12D4CB6AE978E2A4CFBCE27B1203C0DD
:102AC00064E878E29ECFEFEF7E12C8CB8091FC03E2
:102AD0009091FD03A091FE03B091FF0388279C70A5
:102AE000AA27BB272AE0B695A795979587952A959B
:102AF000D1F782309105A105B10571F083309105C0
:102B0000A105B10569F040E00197A105B10511F0FB
:102B100060E008C064E102C044E160E080E003C01E
:102B200044E164E184E10E94672A82E07DC9259640
:102B3000E2E10C94353440E250E0BC0183E00C94B7
:102B400053238091310481608093310408959091E2
:102B50002904937081F0811102C0946007C08D3206
:102B600010F0906B03C0880F880F982B9093290466
:102B700010921F01E6CF089590912904937039F0C7
:102B800080932A0460932B0440932C04DACF089599
:102B9000A7E0B0E0EEECF5E10C941934282E4B01DF
:102BA00080911C010E94BB27392E182F2091000410
:102BB0002983131508F07EC0A12EB12CF501E45035
:102BC000FE4F908180911D01892309F471C05090BE
:102BD0002A0460902B04722C412CC501880F991F88
:102BE000DC01A456BE4FBB83AA83C501880F991F81
:102BF000FC01E356FE4FFD83EC83F9817F1608F05C
:102C000049C0E72CF12CAA81BB81BC91EB2FF0E0ED
:102C1000FF83EE83F701E050FC4F81812E813F81DD
:102C2000281B31093F832E83AC81BD81CC90D12CF0
:102C30008185C81AD108F901EE9F9001EF9F300DF0
:102C4000300D1124CC9CC001CD9C900D900D112411
:102C5000820F931F0E94C62A082F60912D0421E045
:102C6000620F08F46FEFF701EE0FFF1FE050FC4F0B
:102C7000818D928D0E941F2B7C0196014E815F8178
:102C8000652D762D842DF4010995562E672E482E3C
:102C90007394B3CF60912C04842D0E943E2B652D3C
:102CA000762D0E949D2C472F282FC5010E946A2A4D
:102CB0001F5F7FCF81E02FE2231508F480E0279685
:102CC000E2E10C943534A0E0B0E0E9E6F6E10C94E2
:102CD0002334EC0180911C010E94BB27092F182F7F
:102CE00020912D0431E0230F08F42FEF30E040E075
:102CF00050E06FEF7FEF80E090E00E94FD347901BB
:102D0000101708F040C0C12ED12CF601E450FE4F40
:102D1000908180911D018923A1F19091000491502F
:102D200097FD15C0492F092E000C550BFA01E050F4
:102D3000FC4F81891813F3CF440F551FFA01E0505F
:102D4000FC4F218D328D2E153F0548F701C09701AC
:102D500060912D0441E0640F08F46FEFC9010E94F7
:102D60001F2BAC0160912A0470912B0480912C04DC
:102D7000FE0109950E949D2C472F282FC6010E9415
:102D80006A2A1F5FBDCF81E0003308F080E0CDB735
:102D9000DEB7E8E00C943F34A0E0B0E0E2EDF6E10D
:102DA0000C9424348C0180911C010E94BB27EC01FF
:102DB00060912D046695669521E0620F08F46FEF2F
:102DC0008091FC039091FD030E941F2BD82ECD17FC
:102DD000E8F4EC2EF12CF701E450FE4F9081809145
:102DE0001D01892389F060912A0470912B04809140
:102DF0002C042D2D4C2FF80109950E949D2C472F56
:102E0000282FC7010E946A2ACF5FE1CF81E0D0332B
:102E100008F080E0CDB7DEB7E7E00C944034A0E0E6
:102E2000B0E0E5E1F7E10C9420346C0180911C01E5
:102E30000E94BB27192FC82F60912D0466956695B7
:102E40008091FC039091FD030E941F2BD82F80E4FA
:102E50008D0F0E94872A90E8F92EF80E8D2F0E9480
:102E6000872A20E8922E980EC117F8F4AC2EB12CC8
:102E7000F501E450FE4F908180911D01892399F066
:102E800060912A0470912B0480912C04ED2E0C2F5C
:102E9000292D4F2DF60109950E949D2C472F282F93
:102EA000C5010E946A2ACF5FDFCF81E0103308F0AE
:102EB00080E0CDB7DEB7EBE00C943C34A0E0B0E0AE
:102EC000E4E6F7E10C941E345C0180911C010E9441
:102ED000BB27F92E182F60912D0466958091FC0375
:102EE0009091FD030E941F2B782E1F1508F042C001
:102EF000812E912CF401E450FE4F908180911D01B0
:102F00008923B1F1F401EE0FFF1FE456FE4FC0819B
:102F1000D0E0C057D109F401EE0FFF1FE356FE4F7A
:102F2000C080D12C80E2C81AD108CC9F9001CD9FDF
:102F3000300D300D1124CC9CC001CD9C900D900D16
:102F40001124820F931F0E94C62A082F60912A0421
:102F500070912B0480912C04E72C9601AE01F501B1
:102F600009950E949D2C472F282FC4010E946A2A90
:102F70001F5FBBCF81E0FFE2FF1508F480E0CDB713
:102F8000DEB7EDE00C943A34A0E0B0E0EAECF7E113
:102F90000C9423347C0180911C010E94BB27D92E04
:102FA000182F60912D0466958091FC039091FD038C
:102FB0000E941F2BC82E1D1570F5C12FD0E0FE01F9
:102FC000E450FE4F908180911D01892311F1FE0193
:102FD000EE0FFF1FE356FE4F208130E020523109F3
:102FE000FE01EE0FFF1FE456FE4F408150E04057B8
:102FF000510960912A0470912B0480912C040C2DAE
:10300000F70109950E949D2C472F282FCE010E9481
:103010006A2A1F5FD0CF81E0FFE2FD1508F480E04F
:10302000CDB7DEB7E8E00C943F34AAE2B0E0EBE1C4
:10303000F8E10C942834E4EFF3E08091F1008193FF
:1030400043E0EC3FF407C9F78091F503833009F4BE
:1030500063C030F4813071F0823009F4A2C0B9C08D
:103060008A3009F48EC08B3009F46EC0893009F0C3
:10307000B0C020C08091F403813A09F0AAC08091C9
:10308000E800877F8093E8008091F8039091F9032E
:10309000892B21F468E088EE93E003C060E080E0D3
:1030A00090E070E00E94F5228091E8008B77809399
:1030B000E8008FC08091F403813209F08AC08091CA
:1030C000F8039091F903009719F0039709F081C074
:1030D0008091E800877F8093E8008091E80082FD7E
:1030E00005C08091F2038111F8CF73C02091F300E5
:1030F0008091F20090E0922B029731F48091F100E0
:10310000813011F0863021F48091F1008093190113
:103110008091E8008B7759C08091F403813A09F0DF
:1031200058C08091F8039091F903892B09F051C0A0
:103130008091E800877F8093E8008091E80080FF1D
:10314000FCCF80911A013CC08091F403813209F0D8
:1031500040C08091F8039091F903892BD1F58091BB
:10316000E800877F8093E8000E94642181E09091CD
:10317000F603911101C080E080931A010E940D2E88
:1031800028C08091F403813221F58091E800877F87
:103190008093E8000E9464218091F70380931801D6
:1031A00018C08091F403813AA1F48091E800877FF0
:1031B0008093E8008091E80080FFFCCF80911801A7
:1031C0008093F1008091E8008E778093E8000E9460
:1031D00064218091E80083FFF0C18091F403909115
:1031E000F503492F50E04A30510508F0E6C1FA01D5
:1031F000E456FF4F0C946D35803821F0823809F089
:10320000DCC108C08091F0039091F103992389F00B
:1032100082600FC08091F8038F70873008F0CDC1B5
:103220008093E9008091EB0085FB882780F910925C
:10323000E9009091E800977F9093E8008093F10077
:103240001092F1007BC1282F2D7F09F0B6C1882391
:1032500019F0823061F0B1C18091F603813009F03C
:10326000ACC1933009F080E08093F1032EC08091CF
:10327000F60381112AC08091F8038F702FEF280F79
:10328000263008F09AC18093E9002091EB0020FFDE
:103290001CC0933021F48091EB00806214C09091A7
:1032A000EB0090619093EB0021E030E0A90102C0B7
:1032B000440F551F8A95E2F74093EA001092EA0006
:1032C0008091EB0088608093EB001092E900809180
:1032D000E800877F8093E800F7D76FC181116DC147
:1032E0001091F6031F778091E3008078812B809303
:1032F000E3008091E800877F8093E800E5D7809124
:10330000E80080FFFCCF8091E30080688093E300B9
:10331000111102C082E001C083E08093F2034DC12D
:103320008058823008F049C12091F6033091F703AC
:103330002C3D53E0350779F583E08A838AE289835F
:103340004FB7F894DE01139620E03EE051E2E32F00
:10335000F0E050935700E49120FF03C0E295EF7036
:103360003F5FEF708E2F90E0EA3010F0C79601C0FB
:10337000C0968D939D932F5F243149F74FBF809165
:10338000E800877F8093E8006AE270E0CE01019652
:103390000E94F522C1C08091F8039091F903432F58
:1033A000552743305105B1F068F44130510509F417
:1033B00013C14230510509F000C184E790E0E4E711
:1033C000F2E057C04132510589F14232510509F40A
:1033D0003CC0F3C0C901992781309105B9F070F064
:1033E00082309105D9F0039709F0E7C0EAEFF2E0E7
:1033F000E4918E2F90E0EAEFF2E038C0E8E5F3E0E8
:10340000E4918E2F90E0E8E5F3E030C0EEE2F3E0E7
:10341000E4918E2F90E0EEE2F3E028C0E6E1F3E0E5
:10342000E4918E2F90E0E6E1F3E020C08430910536
:1034300008F0C3C0880F991FFC01E05CFE4F0190AB
:10344000F081E02D89E090E014C08430910508F00F
:10345000B4C0FC01EE0FFF1FE85CFE4F0190F0814D
:10346000E02DDC01AC5CBE4F8C9190E0009709F43C
:10347000A4C02091E800277F2093E8002091FA0360
:103480003091FB038217930708F49C0140E021155B
:10349000310589F18091F203882309F43DC085301C
:1034A000D9F18091E80083FD37C08091E80082FD6A
:1034B0002FC08091E80080FFEACF4091F300809117
:1034C000F20090E0942B2115310559F088309105D8
:1034D00040F444914093F100319621503109019616
:1034E000F2CF41E0089709F040E08091E8008E7744
:1034F0008093E800CCCF4111CDCF0AC08091F20378
:10350000882351F0853041F08091E80083FD04C0AC
:103510008091E80082FFF2CF8091E8008B77809362
:10352000E8004BC0803809F048C08091E800877FF0
:103530008093E8008091F3038093F1008091E8008C
:103540008E77C8CE811139C08091F6039091F70330
:103550009927029794F58091E800877F8093E8008F
:103560001091F6031093F303AFD6111106C08091AA
:10357000E30087FD02C081E001C084E08093F20394
:1035800042E061EC81E0BFD642E161EC82E0BBD673
:1035900042E261EC85E0B7D642E261EC83E0B3D66B
:1035A00042E260EC84E0AFD68091F203843011F007
:1035B00081E001C082E080931B018091E80083FFDD
:1035C00010C08091E800877F8093E8008091EB0035
:1035D00080628093EB0005C082E190E0E8EEF2E0CB
:1035E00048CFAA96E3E00C94443480E0089590918B
:1035F000270692FF10C041E0282F2471243009F0E3
:1036000040E031E0282F2871283009F030E04317DE
:1036100011F02CE0822793FF10C041E0282F247185
:10362000243109F040E031E0282F2871283109F0D9
:1036300030E0431711F02CE082273091280630FF4C
:1036400010C051E0282F2171213009F050E041E0F5
:10365000282F2871283009F040E0541711F029E094
:10366000822731FF10C041E0282F2171213109F05C
:1036700040E031E0282F2871283109F030E043176D
:1036800011F029E0822794FD877E08958238910504
:1036900069F1B0F48133910509F475C048F48932B9
:1036A000910509F467C08A32910509F471C0089543
:1036B0008533910509F459C089339105B9F008950E
:1036C000833E910589F138F4803E9105D1F0823E28
:1036D000910529F10895863E9105C9F1873E91052E
:1036E000D9F1843E910509F06CC027C020912706CE
:1036F00020FD57C021FD55C02091280623FD5BC049
:1037000008958091270680FD48C08091280680FF9B
:1037100048C08091270684FD46C083EE51C0809149
:10372000270682FF3CC0F5CF8091270682FD37C077
:103730008091280680FD35C0ECCF8091280681FF5E
:1037400036C08091270684FD2EC087EE39C0809157
:10375000270683FF2AC0F5CF8091270683FD25C069
:103760008091280681FD23C0ECCF8091270685FD3E
:1037700022C01FC08091270685FD1BC080912806AE
:1037800083FF19C00AC08091270686FD16C017C0A6
:103790008091270686FD13C010C089E311C082EE18
:1037A0000FC080EE0DC080E00BC086EE09C084EE35
:1037B00007C085E305C089E203C08AE201C081E356
:1037C00090E0089590919E0480917504892B9091CA
:1037D00074049923E1F0892B90911A01913041F4FE
:1037E0009091270697FF04C09EE12FEA34E003C0C2
:1037F00096E027EA34E0F90120E0915028F0319179
:103800003323D9F32F5FF9CF211110927404089557
:10381000209172049091390457E02917A9F030E003
:10382000529FF001539FF00D1124E65CFB4F718114
:10383000761306C07081781303C07581741306C0B7
:103840002F5F3F4F2770E9CF80E0089581E0089512
:103850007E30B0F46630A0F48330A0F494E5899F04
:10386000F001112486E0789FE00DF11D1124E60F90
:10387000F11DEE0FFF1FE45AFC4F859194910895BE
:1038800080E001C081E090E008951F93CF93DF9323
:10389000FDDEEC01C11580E5D807E8F5C11590E41F
:1038A000D90708F0A6C0C03ED10530F5CD3CD10502
:1038B00008F094C0C83AD10578F4C53AD10508F0AB
:1038C00083C0C130D10509F47CC008F4EBC0C4301A
:1038D000D10508F0EAC0E6C0C33CD10508F0E2C05B
:1038E000C85AD0E0CC0FDD1FC15DDD4F0990D881F3
:1038F000C02DCE019464DAC0C11580E2D80708F06B
:10390000C6C0C11591E0D90708F06BC0C83ED1050B
:1039100008F4CBC0C7C0C03682E5D80728F5C0344C
:1039200092E5D90708F076C0C03282E5D80708F0E2
:1039300069C0C11592E5D90708F47EC04C2F4695A1
:10394000469580E2489FA0011124C37021E030E039
:10395000C90102C0880F991FCA95E2F7EA01C82B76
:10396000D92BCE019D68A2C0C03A82E5D807B8F431
:103970008C2F8F71C03892E5D90708F077C08695F3
:10398000869590E2899F90011124C37081E090E0B8
:1039900002C0880F991FCA95E2F79A6864C0C03CBC
:1039A00082E5D80708F469C0C03E92E5D90708F05F
:1039B00079C0CF71DD27DC2FCC27CE01806F906AD4
:1039C00075C081E090E072C0C55AD0E0C45DDD4FA3
:1039D0008881C82FD0E0CE01906468C0CE01906588
:1039E00065C08D2F04DE182FCE0199274FDE1F7181
:1039F00057C0CE0199274ADECC27DF70D06A8C2BC6
:103A00009D2B54C0CF71D0E0DC2FCC27CE01816F2D
:103A1000906A4CC08C2F8F718695869590E2899F15
:103A200090011124C37081E090E002C0880F991FBB
:103A3000CA95E2F79C6817C08C2F8F71D8DD95E08E
:103A4000D695C7959A95E1F7CF70D0E0DC2FCC27BB
:103A5000282F30E084FF05C084E0220F331F8A95B1
:103A6000E1F7D069CE01822B932B20C090E0D82FB4
:103A7000CC27CE01846F906A19C08C2F8F71B7DD6F
:103A80008F7190E0D82FCC27CE0190620FC08D2F80
:103A90008F71ADDD182FCE019927F8DD1F7190626F
:103AA000912B04C080E090E001C0CE01DF91CF9166
:103AB0001F910895809590919E04892380939E0480
:103AC000089580911A01813061F58091270687FF62
:103AD00028C078DE8093AE0440E250E066E774E0F0
:103AE0008DEA94E00E947335892B09F43EC080E290
:103AF000EDEAF4E0A6E7B4E001900D928A95E1F7D3
:103B0000E0912306F0912406309779F10480F58145
:103B1000E02D309751F186E08093AD048DEA94E07A
:103B200023C050DE8093A50448E050E066E974E0CD
:103B300085EA94E00E947335892BB9F088E0E5EAC4
:103B4000F4E0A6E9B4E001900D928A95E1F7E091E6
:103B50002306F0912406309741F00280F381E02D96
:103B6000309719F085EA94E00995089590917304CF
:103B70008095892380937304282F277069F4981700
:103B800059F09091280692FF07C0869586958695F4
:103B90000E94CC2D1092730408959091280692FBF8
:103BA000222720F9281771F080FB92F990932806BC
:103BB000609127067091280684E090E00E94F93415
:103BC00082E0D4CF089580917204909139048917CE
:103BD00019F08F5F8770FBCF0895CF93DF938091AB
:103BE000380482958F7009F04DC080913704882386
:103BF00009F448C080917204409139045091330413
:103C000060913204C0913404D091350477E0841778
:103C1000C9F190E0789FF001799FF00D1124DF0148
:103C2000A65CBB4F14962C911497222341F1119658
:103C30002C911197251323C02C91261320C0159683
:103C40002C91159721111BC012962D913C91139721
:103C50002C1B3D0B283C310590F4809138048F706B
:103C6000806180933804E05CFB4F80818F708061BD
:103C7000808382E394E00E94A703A5DF03C001963E
:103C80008770C5CFDF91CF910895A4E1B0E0EBE458
:103C9000FEE10C941F348C0186E0F801DE011F96D2
:103CA00001900D928A95E1F7F8018481E58092E315
:103CB000892E94E0992E9091360491111FC088238B
:103CC00009F45FC1EE2009F441C0C8010E94EB2D48
:103CD000F82E8823D9F187E0F801D40101900D92E4
:103CE0008A95E1F780913604813031F48091320475
:103CF000909133040E94522D70DF45C1F801D080AD
:103D0000C180A280B380F0903704209134043091B8
:103D10003504FF2009F4E4C0A501421B530B483CC5
:103D2000510508F09AC0882309F42DC18091380408
:103D3000282F207F90913304222361F09C1509F4F1
:103D40005EC0C8010E94EB2D811161C0C8010E94B4
:103D5000A70317C19C1113C0909132049D110FC08D
:103D6000E1100DC08F7080618093380482E394E08D
:103D70000E94A70380913804F801868300C1E110F6
:103D800038C040E06C2D8D2D43DD40E06C2D8D2D35
:103D90003FDDE82E8111F3C0DF86C88A8F859889C0
:103DA0000E94522D292F22952F70243020F49F70CD
:103DB000223028F009C02A50223080F014C0992304
:103DC00049F0811107C013C0992321F0F8019681B1
:103DD000907F69F0805E883030F409C0803F38F011
:103DE000815F833020F0C8010E94A703EF2CFE2CD6
:103DF000CAC080913804816080933804C0C090911B
:103E000032049D119ECFE1109CCFF80197C0EE20A7
:103E100009F49CCF20913804822F82958F7090E016
:103E200002978CF0809132049091330499878887AF
:103E3000BB86AA86809136048C871D862E87CE018C
:103E400008960E94A70387E0F801A2E3B4E001907E
:103E50000D928A95E1F7C1DE94C090913804292F24
:103E6000207F51F482E394E00E94A70387E0F401ED
:103E700011928A95E9F783C0882309F484C0809160
:103E800033048C110CC0809132048D1108C0E110F4
:103E900006C0F8019683C8010E94A7036AC0C80142
:103EA0000E94EB2D882309F451CFEE2009F44ECF68
:103EB00020913804822F82958F7090E002971CF237
:103EC00080913204909133049A838983BC82AB82BF
:103ED000809136048D831E822F83CE010196B1CF4F
:103EE000A21AB30AF8ECAF16B10408F042C0882356
:103EF00009F447C0FE2CEE2009F428CF809133044A
:103F00008C1129C0809132048D1125C09091380404
:103F100090FD18C0892F82958F70282F30E02115D1
:103F2000310581F0F80196832F30310541F08F5F24
:103F3000982F9295907F86818F70892B8683C801F8
:103F40000E94A70387E0F801A2E3B4E001900D927C
:103F50008A95E1F718C0C8010E94EB2D811173CF3B
:103F600080913804816080933804C8010E94A703BF
:103F70000AC087E0F40111928A95E9F704C0F12C98
:103F800002C0FF24F3948F2D6496ECE00C943B3434
:103F9000EF92FF920F931F93CF93DF9380911001C5
:103FA00090911101892BD1F08091A1048F5F8093B2
:103FB000A104811113C00E941E3290E09093110160
:103FC00080931001892B51F42FEF83EC99E021505D
:103FD00080409040E1F700C00000D3D306E912E032
:103FE000C0E0D0E087E0E82EED0E8D2F0E9450312A
:103FF0008E2D0E9450318D2F0E94AD318F73F801AC
:104000009081891721F08083FF24F39401C0F12C63
:104010008E2D0E94AD318F73F8019781891719F0A9
:10402000878381E001C080E0F82ACF290E9499317E
:10403000DF5F0F5F1F4FD730A9F6CC2351F081E02F
:104040008093A4040DD49093A3048093A204C0E0B1
:1040500023C08091A4048823F9F00091A204109158
:10406000A304FED3801B910B4497B0F04EE050E0C8
:1040700066E972E088EA92E00E947335892B51F07C
:104080008EE0E6E9F2E0A8EAB2E001900D928A95AE
:10409000E1F7C1E01092A4048C2FCDB7DEB7E6E0C3
:1040A0000C944134A6E0B0E0E8E5F0E20C9427344B
:1040B000D7D38C0180919F049091A0040817190711
:1040C00079F019821A82CCD3682F49815A81792FCD
:1040D00080E090E00E9438301093A00400939F0489
:1040E0002696E4E00C944334809119010895A0E0F1
:1040F000B0E0EDE7F0E20C9421348DE5C82E85E0C8
:10410000D82E95E6A92E92E0B92EE12CF12CF601DD
:1041100080818823C1F0C0E0D0E0A7014C0F5D1F73
:1041200043535B4F6C2F6C5DF501808105E010E01F
:1041300020E130E0880F0E942D336096C039D10510
:1041400061F7F6011082F4EACF0ED11C84EAE80E82
:10415000F11CEFEFAE1ABE0AF8E4EF16F1E0FF062D
:10416000B1F6CDB7DEB7EAE00C943D34FF920F9381
:104170001F93CF93DF93182F062FF42EC0E0D0E0CB
:104180002F2D402F612FCE01E4D42196C033D105CD
:10419000B9F7CDB7DEB7E5E00C9442341F920F9229
:1041A0000FB60F9211242F933F934F935F936F930A
:1041B0007F938F939F93AF93BF93CF93DF93EF93AF
:1041C000FF93C091E900CF708091EC00D82FD1709F
:1041D00080FDD0E81092E9008091F000877F809305
:1041E000F00078940E9415181092E9008091F00078
:1041F00088608093F000CD2BCF70C093E900FF91D1
:10420000EF91DF91CF91BF91AF919F918F917F916E
:104210006F915F914F913F912F910F900FBE0F9033
:104220001F901895E8EDF0E080818E7F80831092DA
:10423000E2001092DA001092E100A0EEB0E08C9162
:1042400081608C9380818F77808319BCA7EDB0E06B
:104250008C918E7F8C9380818F7E808310922E062E
:1042600008952091E4003091E50095E64091EC003E
:10427000842F817040FF23C08091E80080FD1DC025
:104280008091F203882399F0853099F08091EB00BA
:1042900085FD11C04091E4005091E50024173507D9
:1042A00029F3915011F09A01E1CF84E0089582E062
:1042B000089583E0089581E0089580E00895409195
:1042C000E80042FFDDCF08958091F40387FF11C01D
:1042D0008091E80082FD05C08091F2038111F8CF42
:1042E00011C08091E8008B770BC08091F203882386
:1042F00049F08091E80080FFF8CF8091E8008E7748
:104300008093E8000895982F973068F59093E9001E
:10431000981739F07091EC002091ED005091F00069
:1043200003C0242F762F50E021FD02C09F5FECCF09
:104330003091EB003E7F3093EB003091ED003D7FFC
:104340003093ED003091EB0031603093EB007093CF
:10435000EC002093ED005093F0002091EE0027FD3B
:10436000E5CF80E008958F708093E90081E00895A3
:10437000A0E0B0E0EEEBF1E20C942334C8EDD0E025
:1043800088818F7E8883E7EDF0E080818160808383
:1043900084E082BF81E080932E0688818E7F8883AF
:1043A00002EE10E0F80110821092DA0081EEC82EC1
:1043B000D12CF601108288818F778883888180686C
:1043C000888388818F7D888319BC1092F2031092B4
:1043D000F3031092F1031092F00390EEE92EF12C0A
:1043E000F70180818B7F808388818160888342E0B0
:1043F00060E080E088DFF60180818E7F8083F801B5
:10440000808181608083808188608083F7018081E2
:104410008E7F8083888180618883CDB7DEB7E8E0B6
:104420000C943F341F920F920FB60F9211242F93CA
:104430003F934F935F936F937F938F939F93AF932C
:10444000BF93EF93FF938091E10082FF09C08091B9
:10445000E20082FF05C08091E1008B7F8093E10044
:104460008091DA0080FF28C08091D80080FF24C0AE
:104470008091DA008E7F8093DA008091D90080FFEE
:1044800016C080E189BD82E189BD09B400FEFDCF7F
:1044900081E08093F20380912E0681110DC0C2DE6F
:1044A00067DF8091E20084608093E20005C019BC60
:1044B0001092F20310922E068091E10080FF1AC044
:1044C0008091E20080FF16C08091E2008E7F809391
:1044D000E2008091E20080618093E2008091D80048
:1044E00080628093D80019BC85E08093F20383E05A
:1044F00080931B018091E10084FF37C08091E2002E
:1045000084FF33C080E189BD82E189BD09B400FE2A
:10451000FDCF8091D8008F7D8093D8008091E100FD
:104520008F7E8093E1008091E2008F7E8093E20095
:104530008091E20081608093E2008091F303882300
:1045400011F084E007C08091E30087FD02C081E0A4
:1045500001C083E08093F2038091F203843011F074
:1045600081E001C082E080931B018091E10083FF24
:104570002BC08091E20083FF27C08091E100877FFC
:104580008093E10082E08093F2031092F303809124
:10459000E1008E7F8093E1008091E2008E7F809326
:1045A000E2008091E20080618093E20042E060E0FE
:1045B00080E0A9DE8091F00088608093F00081E0C7
:1045C00080931B0180931A01FF91EF91BF91AF91EE
:1045D0009F918F917F916F915F914F913F912F911B
:1045E0000F900FBE0F901F9018952091FA033091F5
:1045F000FB032617370748F06115710539F4209140
:10460000E8002E772093E80001C0B901FC0120E00A
:104610006115710579F18091F2038823F1F18530FC
:10462000F1F18091E80083FD3CC08091E80082FDBB
:104630002EC08091E80080FFEBCF2091F3008091A5
:10464000F20090E0922B6115710551F088309105D0
:1046500038F421912093F100615071090196F3CF54
:1046600021E0089709F020E08091E8008E778093A0
:10467000E800CECF2111CFCF0AC08091F20388236A
:1046800061F0853061F08091E80083FD0AC080917F
:10469000E80082FFF2CF80E0089582E0089583E091
:1046A000089581E008950F931F93CF93DF938B01BB
:1046B000EA019091F2039430A1F58F708093E900A4
:1046C0008FEF9091E800815095FD06C095ED9A9589
:1046D000F1F700008111F5CF8091E80085FF21C03E
:1046E000C0DD811115C0209789F08091E80085FD1B
:1046F00006C08091E8008E778093E800F1CFF80142
:1047000081918F018093F1002197EDCF90E001C05E
:10471000982F8091E8008E778093E80081E09111D6
:1047200001C080E0DF91CF911F910F91089543E088
:1047300050E0BC0185E0B7CF45E050E0BC0182E02D
:10474000B2CF40E250E0BC0185E0ADCFCF93DF9324
:10475000EC0148E050E0BC0181E0A5DF88E0FE010B
:10476000A8EEB3E001900D928A95E1F7DF91CF9129
:104770000895603229F4BC0140E250E083E093CF19
:1047800008959AE088E10FB6F894A89580936000A8
:104790000FBE90936000FFCFF89481E08093E0001B
:1047A00080E28093D800E9ECF0E010828FE19EE493
:1047B0000197F1F700C000001DBA109268001CBC00
:1047C00010BE1FBA10927A0010926E0010926F0005
:1047D00010927100109272001082ECEBF0E01082E7
:1047E00014B817B81AB81DB810BA108215B818B88E
:1047F0001BB81EB811BA0C94003F089578941F920C
:104800000F920FB60F9211248F939F93AF93BF9384
:1048100080912A0690912B06A0912C06B0912D062E
:104820000196A11DB11D80932A0690932B06A0939B
:104830002C06B0932D06BF91AF919F918F910F9051
:104840000FBE0F901F9018952FB7F89460912A060D
:1048500070912B0680912C0690912D062FBF089504
:104860002FB7F89480912A0690912B06A0912C06E0
:10487000B0912D062FBF08951F920F920FB60F9281
:1048800011248F939F93AF93BF9380912906811139
:1048900013C080912A0690912B06A0912C06B0910E
:1048A0002D064196A11DB11D80932A0690932B06DB
:1048B000A0932C06B0932D06BF91AF919F918F913D
:1048C0000F900FBE0F901F901895CF93DF93EC01C0
:1048D000C7DF8C1B9D0BDF91CF91089590911A013A
:1048E000913021F49091270697FD03C0E5EAF4E0AA
:1048F0001DC0E82FE695E695E695EE31E0F4F0E090
:10490000E355FB4F877021E030E0A90102C0440F5E
:10491000551F8A95E2F7CA01809592818923828387
:104920000895319654E0EB3AF50729F09281891306
:10493000F8CF1282F6CF089590911A019130D1F4F8
:104940009091270697FF16C0E82FE695E695E69525
:10495000EE3140F5F0E0E355FB4F877021E030E0A9
:10496000A90102C0440F551F8A95E2F7CA0192813E
:10497000892B16C0A7EAB4E0EFEF90E02D918217E3
:1049800089F0EF3F19F4211101C0E92F9F5F9630A4
:10499000A9F7EF3F39F00E2E000CFF0BEB55FB4F44
:1049A000828308950895A3E0B0E0E9EDF4E20C9469
:1049B0002934209125063091260628173907B1F0B1
:1049C0009093260680932506E0912306F091240615
:1049D000309761F00084F185E02D309739F024E0C4
:1049E00029839B838A83CE01019609952396E2E071
:1049F0000C944534A3E0B0E0E0E0F5E20C942934F7
:104A0000209121063091220628173907B1F09093A2
:104A1000220680932106E0912306F0912406309728
:104A200061F00084F185E02D309739F023E029838F
:104A30009B838A83CE01019609952396E2E00C942C
:104A40004534E0912306F0912406309739F0019027
:104A5000F081E02D309711F00995089580E00895D8
:104A6000FFDE20911D06211104C020911E06222385
:104A700021F090931B0680931A0620911F062111A6
:104A800004C020912006222321F0909319068093E0
:104A90001806E0912306F0912406309741F0068035
:104AA000F781E02D309719F08CE196E00995089593
:104AB0008091170680FD18C081FD14C082FD16C0CC
:104AC00080911606882381F08C3380F427E0829F42
:104AD000C00111246CE370E00E945A35862F672BC9
:104AE00019F005C083E0089581E0089587E00895F6
:104AF0008091170680FD17C081FD17C082FD19C087
:104B000080911506882399F08C3398F428E3829FCE
:104B1000C00111246CE370E00E945A35862F672B88
:104B200049F481E008958EE008958CE1089588E0CD
:104B3000089588E30895282F35EB2303C00111243D
:104B400097FF03C08058910902C080589F4F892F5A
:104B50000895A4E0B0E0EFEAF5E20C942634803347
:104B6000910508F049C0122F042FF62EBC01660FE4
:104B7000771F660F771F6C5A7A4F44E050E0CE01E2
:104B800001960E94A534898183702A8130E0682FC4
:104B900070E044EA849FC001112483539B4FFC01C1
:104BA000E20FF31FE0815B814C81EF110CC0FC012F
:104BB000E50FF11DE081E01306C0FC01E40FF11DDB
:104BC00080818117C9F0E4EAE69FC001E79F900D5C
:104BD000112483539B4FFC01E20FF31FF082FC0171
:104BE000E50FF11D0083FC01E40FF11D1083FC01B2
:104BF000E057FF4F21E020832496E5E00C944234F7
:104C0000A1E0B0E0E6E0F6E20C9427344983E82F17
:104C1000F0E0EB59FD4F808105E010E021E030E04D
:104C2000AE014F5F5F4F880F0E942D332196E4E065
:104C30000C944334A4E0B0E0E0E2F6E20C942134BA
:104C40000E94B03210E04BE06DEF812FD9DF40E0E1
:104C50006AE0812FD5DF8FE39CE90197F1F700C06F
:104C6000000040E060E0812FCBDF40E061E0812F79
:104C7000C7DF40E066E0812FC3DF40E06DEF812FAA
:104C8000BFDF00E040E0602F812FBADF0F5F02310D
:104C9000C9F740E0602F812FB3DF0F5F0432C9F7FF
:104CA00040E0602F812FACDF0F5F043BC9F74BE082
:104CB0006DEF812FA5DF41E06AE0812FA1DF40E0A9
:104CC0006DEF812F9DDF1F5F123009F0BCCF04E52F
:104CD00015E094E1C92E96E0D92E24EAA22EEE2406
:104CE000E394F12CBB24B39444E050E0B801CE012E
:104CF00001960E94A5344A813B812C818981837071
:104D0000542F569556955695A89EC001112483534D
:104D10009B4FFC01E50FF11DEF56FF4F4770B701A8
:104D200002C0660F771F4A95E2F7AB015081452B11
:104D30004083432F469546954695FC01E40FF11DAF
:104D4000EF56FF4F3770A70101C0440F3A95EAF7BD
:104D50003081432B4083322F369536953695FC01B2
:104D6000E30FF11DEF56FF4F2770A70102C0440F5C
:104D7000551F2A95E2F79A013081232B2083FC01ED
:104D8000ED55FF4FB0820C5F1F4FC016D10609F0E2
:104D9000ABCF8DECC82E84E0D82EF12C560153EA0F
:104DA000A50EB11CF5018081882391F000E010E090
:104DB000F801EF56FF4FEC0DFD1D4081602F8F2D48
:104DC0001FDF0F5F1F4F0231110591F7F5011082B0
:104DD000F394F4EACF0ED11C42E0F412DFCF249614
:104DE000EAE00C943D341F93CF93DF93C82FD0E0BB
:104DF000FE01E450FE4F8081682371F0A9D3182F83
:104E000080E8BBD37FE7780F612F80912C0495D584
:104E1000472F282FCE015ED3DF91CF911F910895A8
:104E2000A0E0B0E0E6E1F7E20C942434C82FD0E033
:104E3000FE01E450FE4F8081682329F1D0902B04BD
:104E400000912C0410912A04E12EF12C83E095D3DB
:104E5000282FC7018C549F4F68E671E00E945A3595
:104E60008E199F0997FD039695958795959587953A
:104E7000612F289F600D11247D2D802F5ED5472F37
:104E8000282FCE0127D3CDB7DEB7E7E00C9440340E
:104E9000E9E2F4E0248130E1231B08F420E02483DC
:104EA0000C94A115E9E2F4E0248130E1230F08F429
:104EB0002FEF24830C94A115E9E2F4E0438120E173
:104EC000421B08F440E08181628190E00C94BC15A3
:104ED000E9E2F4E0438120E1420F08F44FEF8181E1
:104EE000628190E00C94BC15E9E2F4E0628120E17B
:104EF000621B08F460E08181438190E00C94BC1552
:104F0000E9E2F4E0628120E1620F08F46FEF818151
:104F1000438190E00C94BC15E9E2F4E0818190E0DB
:104F20004381628108970C94BC15E9E2F4E0818129
:104F300090E04381628108960C94BC15809129040D
:104F400086958695815009F48CE20C94A715809182
:104F50002904869586958F5F8D3208F081E00C9448
:104F6000A715E9E2F4E0908181E08927808310921F
:104F70001F010C94A11594E0899F800D112495E0E8
:104F8000980F913308F090E308954F925F926F92DB
:104F90007F928F929F92AF92BF92CF92DF92EF92C9
:104FA000FF92CF938090580690905906A0905A0691
:104FB000B0905B0649DC6B017C01C818D908EA088F
:104FC000FB0842DC4B015C01609358067093590664
:104FD00080935A0690935B06A0912F06EFE2F6E0CD
:104FE0008A2F90E04FEF5FEF60E070E04C195D09B1
:104FF0006E097F09A91799F0218D328D2901612C45
:10500000712C441555056605770510F4815004C0D0
:105010002C0D3D1D328F218F9F5F3296EBCF8093F9
:105020002F0680915C06811108C0C09129048C2F45
:10503000837019F0C695C69501C0C0E080911F012C
:105040008130D9F028F0823011F1833061F14EC007
:1050500010921C018092FC039092FD03A092FE032B
:10506000B092FF0389E2EFE2F6E0A0E0B4E0019045
:105070000D928A95E1F781E013C08C2F0E94A50E56
:10508000CC23A1F180911C01815075DF2FC0C0930A
:1050900021018091290483708093200128D883E026
:1050A00080931F0123C080913104882351F048E090
:1050B00050E067E170E089E294E00E94D034109201
:1050C0003104C090FC03D090FD03E090FE03F0900B
:1050D000FF03BADBDC01CB018C199D09AE09BF09C6
:1050E0004A97A105B10510F010921F01CF91FF90D2
:1050F000EF90DF90CF90BF90AF909F908F907F9078
:105100006F905F904F900895EF92FF920F939701E9
:10511000201B31092F3F310519F010F02FEF30E03F
:105120002095382F320F08F43FEF832F0F91FF9017
:10513000EF900895EF92FF920F939701201B310992
:105140002F3F310519F010F02FEF30E0322F30955E
:10515000482F430F08F44FEF842F620F0F91FF90F9
:10516000EF900895EF92FF920F93972F093438F440
:10517000B701601B71096F3F710519F010F06FEFF7
:1051800070E0485F5F4F4131510540F0A901485F31
:105190005F4F4131510510F06FEF70E06095482F7F
:1051A000460F08F44FEF842F37FF02C02D5F3F4FAB
:1051B000359527953595279560912A04620F792FAB
:1051C0000F91FF90EF900895EF92FF920F93E00EF2
:1051D000F11CF90137FF03C0F195E195F10924E0D5
:1051E000EE0FFF1F2A95E1F7EF3FF10519F014F0DC
:1051F000EFEFF0E09A0157FF03C031952195310997
:1052000094E0220F331F9A95E1F72E173F070CF415
:10521000F901EE0DFF1DEF3FF10519F010F0EFEF72
:10522000F0E02E2F2095382F320F08F43FEF832F18
:105230000F91FF90EF900895EF92FF920F939701D7
:1052400095E0099F200D311D11242F3F310519F0E4
:1052500010F02FEF30E02095382F320F08F43FEF99
:10526000832F0F91FF90EF9008950F931F9310E0FD
:10527000F801EE0FFF1FE456FE4F9081905797FD07
:105280009195000F111FF801E356FE4FE081F0E009
:10529000B097DF01AA0FBB1F8D010E0F1F1F200348
:1052A000D001219FB00D1124E8E3F0E0E91BF109E2
:1052B00097FDF3959F01220F331F89010E0F1F1FCA
:1052C00040039001419F300D11242A0F3B1F37FFEF
:1052D00002C021583F4F220F232F221F330B620F92
:1052E0001F910F9108950F931F93522F10E0F80113
:1052F000EE0FFF1FE356FE4FE081F0E0B097EE0F98
:10530000FF1F9F015203D001539FB00D1124000FC6
:10531000111FF801E456FE4F008110E000571109FB
:10532000000F111F40039001419F300D11242A0FDF
:105330003B1F37FF02C021583F4F220F232F221F50
:10534000330B620F1F910F9108950F931F93522FEC
:1053500010E0F801EE0FFF1FE356FE4FE081F0E092
:10536000B0979F015203D001539FB00D1124000F3D
:10537000111FF801E456FE4F008110E0005711099B
:1053800040039001419F300D11242A0F3B1F37FF2E
:1053900002C021583F4F220F232F221F330B620FD1
:1053A0001F910F910895EF920F931F9393E0099F20
:1053B00080011124159507956E2D600F1F910F9197
:1053C000EF900895A22F50E0FA01EE0FFF1FE35671
:1053D000FE4F9081905297FD9195440F551FFA0111
:1053E000E456FE4F3081232F30E02A1B3109290F6C
:1053F000311D97FD3A95620F0895E42FF0E0EE0F0E
:10540000FF1FE356FE4F6081621B0895E42FF0E01A
:10541000EE0FFF1FE456FE4F6081621B0895622F5E
:105420000895FC019B01009721F477FF2BC080E8D1
:105430000895AC0197FF04C044275527481B590B1A
:10544000B901640F751F37FD0CC0241B350BC90152
:10545000A5E0880F991FAA95E1F70E945A3580E2CE
:105460000CC0CB0165E0880F991F6A95E1F7BA017E
:10547000621B730B0E945A3580E6861BF7FF03C040
:105480008195089580E00895EF920F93CF93DF9375
:10549000D72FC82FC9010E19BA01C3DF602F681BAF
:1054A0007D2F8C2FDF91CF910F91EF9008950F9367
:1054B000CF93DF93D72FC82FC901BA01B2DF682F6E
:1054C000600F7D2F8C2FDF91CF910F9108950C9459
:1054D000B62008953ECB0895E9E2F4E085E38083A9
:1054E0008091240190912501A091260181839283CE
:1054F000A3838FE784838FEF858348E050E067E1E3
:1055000070E0CF010E94D034109231040895482FEA
:10551000982F46FD9095E92FEF739F7046FD9F5F92
:10552000E295EF70EE0FF0E0E959FD4F2181299FE0
:10553000802D212D112482958F702295207F822B22
:105540003081982F930F892F47FD819580580895BA
:10555000409122015091230125E038E0429FC00193
:10556000439F900D529F900D1124875E994C90930C
:10557000230180932201890F0895CF93C82FE8DF7C
:105580008C9FC0011124892FCF910895BC018230D6
:10559000910508F40895613E8EE1780748F49B0177
:1055A00095E0369527959A95E1F748E0420F01C0BE
:1055B0004FEF91E0242F30E0290F311D35952795CD
:1055C000229FF001239FF00DF00D11246E177F072D
:1055D00018F44FEF420F04C02F3F39F091E0920FC3
:1055E000491740F78FEF890F08958FEF08950F93B4
:1055F000CF93DF93D72FC82F47FD4195E8E3F0E025
:10560000CF01841B910947FD9395889FB001899F25
:10561000700D700D1124229FC001239F900D900DDD
:105620001124860F971FB2DF682F660F860F682F31
:10563000600F7D2F8C2FDF91CF910F91089520E087
:1056400030E0869F080E211D969F200D311D1124EC
:10565000290F311DC901089520912D0430E1230F38
:1056600008F42FEF60E1822F90E0E9DFBC0188EBC6
:105670009BE00E94053480E090E00895282F269F4B
:10568000020E20E0211D1124822F08951F93CF9335
:10569000DF93C62F172FD82F60E4842F8095EEDF7D
:1056A000682F6C0F712F8D2FDF91CF911F9108956F
:1056B000CF93DF93D62FC72F682F81E0841BDEDFC7
:1056C0006D2F7C2FDF91CF9108951F93CF93DF93A0
:1056D000C62F172FD82FE42FF0E0EE0FFF1FE45650
:1056E000FE4F8081821B87FD819568E1C7DF682FAF
:1056F0006C0F712F8D2FDF91CF911F9108950F9314
:105700001F93CF93DF93D62F072F182FC42F822FED
:10571000FEDEEC2FF0E0EE0FFF1FE456FE4F90810F
:105720009058890F87FD81956CE0880FA7DF682F5F
:105730006D0F702F812FDF91CF911F910F910895E1
:105740001F93CF93DF93C62F172FD82F822F8695C5
:10575000DEDE805887FD81956CE0880F8FDF682F33
:105760006C0F712F8D2FDF91CF911F910895EF92C4
:105770000F931F93CF93DF93162FD72FC82FC901F5
:105780000E190C0FBA014DDE6C2F081B802F76DF2F
:10579000612F7D2FDF91CF911F910F91EF90089591
:1057A000EF920F931F93CF93DF93162FC72FD82F0E
:1057B000C9010E19070FBA0134DE6C2F081B802FA8
:1057C0005DDF612F782F8D2FDF91CF911F910F918A
:1057D000EF9008950F931F93CF93DF93162FD72F3A
:1057E000C82FC9012C2F201B022FBA011ADE982FB7
:1057F000990F890F6C2F081B802F40DF612F7D2FA1
:10580000DF91CF911F910F9108950F931F93CF9325
:10581000DF93162FC72FD82FC901272F201B022F48
:10582000BA01FFDD982F990F890F6C2F081B802F6D
:1058300025DF612F782F8D2FDF91CF911F910F9151
:1058400008950F931F93CF93DF93162FD72FC82F51
:10585000022FE42FF0E0EE0FFF1FE456FE4F64EE40
:1058600080810CDF4C2F50E0282F30E0245E3F4F2A
:10587000201B310937FF03C031952195310983E0A1
:10588000220F331F8A95E1F7CA01821B930B97FF02
:1058900002C080E090E06C2FF1DE612F7D2FDF9160
:1058A000CF911F910F9108950F931F93CF93DF9383
:1058B000162FC72FD82F022FE42FF0E0EE0FFF1F77
:1058C000E456FE4F64EE8081D9DE4C2F50E0282F45
:1058D00030E0245E3F4F201B310937FF03C0319574
:1058E0002195310983E0220F331F8A95E1F7CA0120
:1058F000821B930B97FF02C080E090E06C2FBEDE0E
:10590000612F782F8D2FDF91CF911F910F910895E7
:105910001F93CF93DF93D62FC72F182F822F8695F3
:10592000F6DD805887FD8195612F880FA7DE6D2FEA
:105930007C2FDF91CF911F910895A0E0B0E0E2EAC3
:10594000FCE281C77B01E82FF0E0F11006C0EC5EBD
:10595000F94F8491782F682F72C02F2D30E0EC5EC4
:10596000F94FE491FE2F0E2F10E046E0649FC00136
:105970001124CFEFD0E0BE0148D7AB016BEA64033E
:10598000C001659F900D11248E0D911D8E0D911DEE
:10599000982F990F980FBE01621B730B609FD00167
:1059A000619FB00D709FB00D11248B2FF99EB00137
:1059B0001124672F77277E01E61AF70AB701609F47
:1059C0007001619FF00C709FF00C11246E01C91AD8
:1059D000D108C29EB001C39E700DD29E700D1124DD
:1059E000272F3327C21BD30BC09F9001C19F300DBF
:1059F000D09F300D1124732F4230510591F048F49F
:105A000041155105D9F041305105B1F47E2FEF2DEC
:105A100015C04430510561F040F04630510571F039
:105A20000BC0EB2F832F7F2F09C07F2DEB2F02C0E0
:105A3000E32F7B2F8F2F02C07B2F8F2D6E2FCDB7A3
:105A4000DEB7E8E01CC7CF92DF92FF920F931F935F
:105A5000CF93DF936C010091C7028091C602082B9F
:105A6000C7E0D0E010E0C8010C2E02C095958795E4
:105A70000A94E2F780FD04C02197A8F7F12C09C031
:105A8000FC2EB6018C2F0E94281C0E94451C0197F9
:105A900099F38F2DDF91CF911F910F91FF90DF90A0
:105AA000CF900895CF93DF93EC01CDDFBE010E942C
:105AB000281C0E94451CDF91CF910895292F9E300C
:105AC00078F5863068F590E036E0239F800D911DD3
:105AD0001124682F677023E0969587952A95E1F742
:105AE000FC01EE0FFF1FE80FF91FE35AF94F40E0EA
:105AF00050E080E0219130E0062E02C036952795D7
:105B00000A94E2F721703327042E01C0220F0A9471
:105B1000EAF7822B4F5F5F4F4330510559F70895E5
:105B200080E00895292F9E3088F5863078F590E042
:105B300036E0239F800D911D1124282F277051E0FE
:105B400001C0550F2A95EAF723E0969587952A9587
:105B5000E1F7FC01EE0FFF1FE80FF91FE35AF94FC1
:105B600020E030E070E04081CB01022E02C096952B
:105B700087950A94E2F7817081958427852384278D
:105B800081932F5F3F4F2330310569F7089550D33C
:105B90002ED38093C702089521E030E001C0220F88
:105BA0008A95EAF720958091C7028223F0CF21E001
:105BB00030E001C0220F8A95EAF78091C702822B5C
:105BC000E6CFCF93C82F8091C7028C2B31D3C093DF
:105BD000C602CF910895FC0124812223D1F0808157
:105BE000918160DF92959F70963079F010F4925019
:105BF00001C09A50923068F4803F69F018F4883EF2
:105C000040F409C0843F29F406C0883E20F0813F5B
:105C100011F080E0089581E0089510929E04809133
:105C20001A01813041F48091270687FF04C08EE17C
:105C3000EFEAF4E003C086E0E7EAF4E0DF011D925A
:105C40008A95E9F780E090E00E94FA2480E090E0F5
:105C50000E94D324109275040E94611DECE1F6E0CD
:105C600085E0DF011D928A95E9F7109215061092E2
:105C70001606109217060C943025882341F0809563
:105C8000909175048923809375040C94611D089587
:105C9000882339F090917504892B809375040C94B6
:105CA000611D0895882321F00E945A1D0C94611DE6
:105CB0000895882339F090919E04892B80939E0447
:105CC0000C94611D0895662309F45CC08D3C21F499
:105CD0000E947825819504C08E3C29F40E94782585
:105CE00080931E06C5C08F3C21F40E9478258195C3
:105CF00004C0803D29F40E94782580931D06B8C019
:105D0000893D19F40E94582505C08A3D31F40E944E
:105D10005825819580931F06ABC08B3D21F40E94CE
:105D20005825819504C08C3D29F40E945825809304
:105D300020069EC09FE2980F983078F421E030E072
:105D4000A90102C0440F551F9A95E2F7CA0190912C
:105D50001C06892B80931C068BC08D3D21F48091FD
:105D6000170681600CC08E3D21F480911706826079
:105D700006C08F3D09F07CC0809117068460809337
:105D8000170676C08D3C39F490911E0697FF35C0FA
:105D900010921E0659C08E3C29F490911E061916C9
:105DA000BCF32BC090911D068F3C29F497FF25C0B2
:105DB00010921D0649C0803D19F41916CCF31DC080
:105DC00090911F06893D29F41916BCF410921F0604
:105DD0003BC08A3D19F497FF10C0F8CF8B3D39F4D2
:105DE0009091200697FF09C0109220062DC08C3D8F
:105DF00021F4909120061916BCF39FE2980F983079
:105E000080F421E030E0A90102C0440F551F9A95AB
:105E1000E2F7CA01809590911C06892380931C06A5
:105E200013C08D3D21F4809117068E7F0BC08E3DEF
:105E300021F4809117068D7F05C08F3D29F4809154
:105E400017068B7F8093170680911D06811106C06F
:105E500080911E06811102C01092150680911F06C6
:105E6000811106C080912006811102C01092160691
:105E70000C943025882361F19CEF980F913A18F427
:105E80000E946E240DC090E2980F983058F48770ED
:105E900091E001C0990F8A95EAF7892F0E945A1D57
:105EA0000C94611D9BE5980F933020F480E090E006
:105EB0000C94FA2498E5980F9B3120F480E090E050
:105EC0000C94D32493E3980F933110F460E0FBCE4D
:105ED0000895CF93882309F46DC0C82F8CEF8C0FE1
:105EE000813AA0F580911A018130E1F48091270672
:105EF00087FF18C0EC2FE695E695E695F0E0E355B0
:105F0000FB4F8281282F30E04C2F477081E090E0DA
:105F100002C0880F991F4A95E2F782239323892BA9
:105F200061F410C0E7EAF4E08DEA94E02191C21731
:105F300021F08E179F07D1F705C08C2F0E946E2489
:105F40000E94611D8C2F0E949C2410C080E28C0F47
:105F5000883078F4C77081E090E001C0880FCA955E
:105F6000EAF790919E04892B80939E040E94611D04
:105F700021C0EBE5EC0FE33040F4F0E0E45DFD4FD1
:105F8000808190E00E94FA2415C0E8E5EC0FEB3127
:105F900050F4F0E0EE0FFF1FE15DFD4F8081918135
:105FA0000E94D32407C083E38C0F833118F461E08F
:105FB0008C2F89DECF91089590E0FC01ED57FD4FC5
:105FC000208121111AC0F894FC01EB58FD4F80810B
:105FD000E82FE295EF70F0E031A1282F2F7081E0DB
:105FE00090E001C0880F2A95EAF7982F90959323A7
:105FF00091A392A1892B82A378940895982F9295CA
:106000009F7019F0892F24E001C020E0982F969509
:10601000969511F02E5F892F982F969509F02F5F96
:10602000822F0895A6E0B0E0E7E1F0E311C426E096
:10603000FC01DE01119601900D922A95E1F7FC0119
:10604000258189819A81222349F0662339F0FBDC7E
:10605000182F682F89819A8165DD02C02FDD182FE6
:1060600069817A81812F0E94281C2696E3E00CC466
:10607000A4E3B0E0EDE3F0E3EAC34FA758AB69ABAC
:106080007AAB8BAB9CAB9111109275048E01085DBD
:106090001F4F87E0D8011D928A95E9F786E0FE013F
:1060A000BF96D80101900D928A95E1F78CA58823BF
:1060B000D9F061E0C801B6DF8091C802882389F079
:1060C0008DA5811102C087E001C086E0898388A583
:1060D0008A8389A58B838EEF8C83CE0101960E94E3
:1060E0009B1561E0C8019EDF87E0FE01B896DE01E6
:1060F000919601900D928A95E1F7CE0181960E94CA
:10610000451E81112CC087E0FE01B196DE0111967B
:1061100001900D928A95E1F76DA1662301F120911E
:10612000390430E0C90101968770992740917204C3
:1061300050E08417950761F16D8397E0929FD0013D
:10614000939FB00D1124A65CBB4FFE0131960190C8
:106150000D929A95E1F7809339040E94E31D17E0B0
:1061600080917204909139048917F1F0189FC00151
:106170001124865C9B4F0E94451E8823A9F08091C4
:10618000720490E001968770992780937204E8CF9B
:1061900044DD1092390410927204E2E3F4E087E0E7
:1061A000DF011D928A95E9F7E496E4E06CC335DDE2
:1061B0002FEF84E39CE0215080409040E1F700C045
:1061C0000000089527982F982F98089526982E98C4
:1061D0002E98089525982D982D980895279A2F9AEE
:1061E0000895269A2E9A0895259A2D9A0895CF9368
:1061F000DF93D82F03DFC82F5E98ECDFE7DFE2DF05
:106200008C2F90E0FC013197E730F10568F4EA55F6
:10621000FF4F63C4E9DF08C0E7DFE3DF05C0E4DF69
:1062200002C0E2DFDEDFDADF8D2FDF91CF9108954C
:10623000A0E2B0E0EDE1F1E30BC3182F8091C802BA
:106240008823D9F08091C602812BD8DE90917F06F9
:10625000891799F080937F068FE39CE90197F1F706
:1062600000C0000085E0898380917F068A838EEFDD
:106270008B83CE0101960E949B15812FA096E3E0AF
:1062800003C3A0E2B0E0E6E4F1E3E3C29FEF998349
:106290008A83CE0101960E949B15A096E2E0F5C28A
:1062A000A1E0B0E0E5E5F1E3D2C28730F0F420915F
:1062B000100130911101232BC9F521E030E0A90133
:1062C00002C0440F551F8A95E2F7CA018095898361
:1062D0000AE010E0AE014F5F5F4F62E180E4BDD1A4
:1062E000909311018093100121C090E0FC01ED57C3
:1062F000FD4F208121111AC0F894FC01EB58FD4F8D
:106300008081E82FE295EF70F0E031A1282F2F7007
:1063100081E090E001C0880F2A95EAF7932F982B2F
:1063200091A392A18095892382A378942196E4E099
:10633000AAC20F931F93CF930AE812E0C7E0F801B7
:1063400081918F01811102C08C2F36DECF5FCE305C
:10635000B1F7CF911F910F910895A1E0B0E0E2EB6A
:10636000F1E375C2082F8730C0F48091100190913D
:106370001101892BD1F519820AE010E021E030E00B
:10638000AE014F5F5F4F63E180E4AFD190931101A5
:10639000809310018981809529C082DFAFE6B2E049
:1063A00020E030E010E051E04D91E42FE295EF70F5
:1063B000F0E080A190E04F7002C0959587954A95D6
:1063C000E2F780FD07C0852F022E01C0880F0A94D6
:1063D000EAF701C080E0182B2F5F3F4F26303105D0
:1063E00019F7802FE9DD812F01C080E02196E4E0DC
:1063F0004AC2CF93DF93AFE6B2E045E752E061E0F7
:1064000070E0F8948D91E82FE295EF70F0E021A113
:106410008F70EB0102C0CC0FDD1F8A95E2F7CE0131
:106420009C2F9095922391A392A1892B82A378947B
:106430004A175B0731F7DF91CF910895A2E0B0E0F2
:10644000E3E2F2E304C280E290E0909311018093D2
:10645000100180917E0681110DC082D081E0809371
:106460007E062FEF83ED90E3215080409040E1F7CE
:1064700000C0000019828FE38A830AE010E022E066
:1064800030E0AE014F5F5F4F60E080E4E6D0909374
:10649000110180931001892B61F422E030E0AE01FC
:1064A0004F5F5F4F6CE080E4D8D0909311018093F0
:1064B0001001809110012296E4E0E5C1EF92FF9275
:1064C0000F931F93CF93DF93182FEB011092BC0013
:1064D00084EA8093BC000E9430247C018091BC003F
:1064E00087FD0DC0CF3F8FEFD807C1F3C7010E94D2
:1064F0006524C817D90790F78EEF9FEF2DC08091C4
:10650000B900887F883041F08091B900887F803160
:1065100019F08FEF9FEF20C01093BB0084E88093A9
:10652000BC000E9430248C018091BC0087FD0BC010
:10653000CF3F8FEFD807C1F3C8010E946524C81769
:10654000D90790F7D9CF8091B900887F883111F0B1
:106550008034F9F680E090E0CDB7DEB7E6E091C197
:106560001092B9008CE08093B80008950F931F93A8
:10657000CF93DF93EB018093BB0084E88093BC0052
:106580000E9430248C018091BC0087FD0DC0CF3F5C
:106590008FEFD807C1F3C8010E946524C817D90737
:1065A00090F78EEF9FEF0CC02091B900287F81E01B
:1065B00090E0283211F480E090E091958195910966
:1065C000DF91CF911F910F9108950F931F93CF9358
:1065D000DF93EC0184EC8093BC000E9430248C019A
:1065E0008091BC0087FD0DC0CF3F8FEFD807C1F36E
:1065F000C8010E946524C817D90790F78EEF9FEF56
:1066000003C08091BB0090E0DF91CF911F910F916B
:1066100008950F931F93CF93DF93EC0184E8809349
:10662000BC000E9430248C018091BC0087FD0DC00D
:10663000CF3F8FEFD807C1F3C8010E946524C81768
:10664000D90790F78EEF9FEF03C08091BB0090E0D9
:10665000DF91CF911F910F910895A0E0B0E0E2E3A8
:10666000F3E3EBC0682E762E5A0169010E943024B4
:106670004C010431110550F00F3F8FEF180749F01E
:10668000C80164E170E0C1D0EB0105C0C1E0D0E019
:1066900002C0C5E0D0E0BE01862D10DF7C0197FF6F
:1066A0000BC00F3F8FEF1807B1F3C4010E946524A0
:1066B0000817190780F711C0B801872D57DF7C0133
:1066C000E501CA0CDB1CCC15DD0539F0F7FC05C073
:1066D000B80189914BDF7C01F6CF84E98093BC003F
:1066E000C701CDB7DEB7EEE0C4C0A0E0B0E0EAE796
:1066F000F3E3A3C0782E662E7A01E9010E943024CC
:106700005C010431110550F00F3F8FEF180751F075
:10671000C80164E170E079D06B0107C0CC24C39458
:10672000D12C03C025E0C22ED12CB601872DC6DEA8
:106730004C0197FF0BC00F3FEFEF1E07B1F3C501F0
:106740000E9465240817190780F728C0B801862D14
:106750000DDF4C0197FD22C0F72DF1607F2E0E94C6
:1067600030245C010431110518F10F3F8FEF180739
:1067700019F1C80164E170E048D06B01B601872DC2
:106780009DDE4C0197FD1CC067012197C6018E1943
:106790009F098C179D0750F597FE1DC084E98093D3
:1067A000BC00C4011816190664F580E090E029C009
:1067B000CC24C394D12CE2CF85E0C82ED12CDECFDF
:1067C0000F3FEFEF1E07D1F2C5010E9465240817A5
:1067D0001907A0F6D9CFC801F8DE4C0197FD02C019
:1067E000F6018083FFEFCF1ADF0AD0CF97FCD6CF18
:1067F000C8010FDF4C0197FDD1CFCE0DDF1D88837F
:10680000CDCFCDB7DEB7EEE034C0AA1BBB1B51E144
:1068100007C0AA1FBB1FA617B70710F0A61BB70B10
:10682000881F991F5A95A9F780959095BC01CD01B5
:1068300008952F923F924F925F926F927F928F9224
:106840009F92AF92BF92CF92DF92EF92FF920F93FF
:106850001F93CF93DF93CDB7DEB7CA1BDB0B0FB609
:10686000F894DEBF0FBECDBF09942A8839884888C6
:106870005F846E847D848C849B84AA84B984C8845C
:10688000DF80EE80FD800C811B81AA81B981CE0F53
:10689000D11D0FB6F894DEBF0FBECDBFED01089538
:1068A0008F929F92AF92BF92CF92DF92EF92FF9220
:1068B000CF93DF93EC01688179818A819B81611597
:1068C00071058105910521F464E279ED8BE597E08E
:1068D0002DE133EF41E050E090D049015A019B0196
:1068E000AC01A7EAB1E4A5D06B017C01ACEEB4EF3A
:1068F000A5019401AAD0DC01CB018C0D9D1DAE1D1C
:10690000BF1DB7FF03C00197A109B04888839983D1
:10691000AA83BB839F77DF91CF91FF90EF90DF90A9
:10692000CF90BF90AF909F908F900895B9CF80E0A7
:1069300091E0B6CFA0E0B0E0809300019093010118
:10694000A0930201B09303010895FB01DC0102C092
:1069500005900D9241505040D8F70895DC01CB01CD
:10696000FC01F999FECF06C0F2BDE1BDF89A31965F
:1069700000B40D9241505040B8F70895F999FECFF8
:1069800092BD81BDF89A992780B50895A6E1B0E03F
:1069900044E050E0E5CFA8E1B0E042E050E0E0CFD5
:1069A000DC01A40FB51F4150504040F0CB01840FD3
:1069B000951F2E9105D041505040D8F70895262FAD
:1069C000F999FECF92BD81BDF89A019700B40216E5
:1069D00039F01FBA20BD0FB6F894FA9AF99A0FBE93
:1069E00008950396272FECDFEADF252FE9DF242F18
:1069F000E7CF0196272FE4DFE2CF052E97FB16F4B1
:106A000000940FD057FD05D024D007FC02D046F4E7
:106A100008C050954095309521953F4F4F4F5F4F9F
:106A2000089590958095709561957F4F8F4F9F4FFA
:106A3000089531D0A59F900DB49F900DA49F800D17
:106A4000911D11240895B7FFF4CFF3DF821B930B40
:106A50000895A1E21A2EAA1BBB1BFD010DC0AA1F9F
:106A6000BB1FEE1FFF1FA217B307E407F50720F0B7
:106A7000A21BB30BE40BF50B661F771F881F991F32
:106A80001A9469F760957095809590959B01AC017B
:106A9000BD01CF010895A29FB001B39FC001A39F84
:106AA000700D811D1124911DB29F700D811D112447
:106AB000911D089597FB072E16F4009406D077FDDC
:106AC00008D0A3DE07FC05D03EF4909581959F4F3A
:106AD0000895709561957F4F0895EE0FFF1F059003
:106AE000F491E02D0994FB01DC0104C08D9101902B
:106AF000801921F441505040C8F7881B990B089524
:106B0000FB01DC0102C001900D9241505040D8F7CA
:066B10000895F894FFCF88
:106B1600010000007420A623A1239C239723B923F8
:106B260020003100310031000000010000FF0003A9
:106B3600FFFF390500FFFF394234334F2F42347AC5
:106B4600676751004422476D30020E02C7015A01A1
:106B560086029F02BF02D802FFFFFFFFFFFF1C2134
:106B6600262B2FFF1B20252A2EFF1A1F24292DFF37
:106B7600191E23282CFF181D2227FFFFFFFFFFFFEA
:106B8600FFFFFFFFFFFFFFFF00050A0FFFFF0106E4
:106B96000B1014FF02070C1115FF03080D1216FF48
:106BA60004090E1317FFFFFFFFFFFFFF89009A007E
:106BB600AC00BD00CE00890C9A0CAC0CBD0CCE0C02
:106BC60089199A19AC19BD19CE1989269A26AC26A7
:106BD600BD26CE269A33AC33BD33CE3356004400A1
:106BE600330022001100560C440C330C220C110CFD
:106BF60056194419331922191119562644263326D3
:106C06002226112644333333223311330404040479
:106C1600040404040404040404040404040404042E
:106C2600010101010404040404040404040404042A
:106C3600040404040404040401010101818283E2C2
:106C460000E900EA00B500B600B700CD008301CC2C
:106C5600008A0192019401210223022402250226C0
:106C66000227022A02B300B4006F0070009F01CB16
:106C7600019F02A0027477003131295A1B750AF070
:106C8600F1F4F5F6F7000000000000003031323371
:106C9600929366010101010101010000000000005C
:026CA6000000EC
:00000001FF
